:100000009DC10000CCC10000CAC10000C8C10000F1
:10001000C6C10000C4C10000C2C10000C0C10000D0
:10002000BEC10000BCC10000BAC10000B8C10000E0
:10003000B6C10000B4C10000B2C10000B0C10000F0
:10004000AEC100000C94323DAAC10000A8C100005E
:100050000C94603DA4C10000A2C100000C945E3C61
:100060009EC100000C94283C0C94FE3B98C10000FB
:1000700096C1000094C1000092C1000090C1000030
:100080000C94043D8CC100008AC1000088C10000AE
:1000900086C1000084C1000082C1000080C1000050
:1000A0007EC100007CC100000C94D63C78C10000E9
:1000B00076C1000074C1000072C100000C94A83C1D
:1000C0006EC100006CC100006AC1000068C1000080
:1000D00066C1000064C1000062C1000060C1000090
:1000E0005EC100004E414E494E495459494E46CDDD
:1000F000CCCC3D0AD7233C17B7D13877CC2B3295DF
:1001000095E6241FB14F0A000020410000C84200BC
:10011000401C4620BCBE4CCA1B0E5AAEC59D740086
:10012000407A10F35A00A0724E18090010A5D4E8C6
:100130000000E87648170000E40B54020000CA9A59
:100140003B000000E1F505000080969800000040AB
:10015000420F000000A086010000001027000000F0
:1001600000E803000000006400000000000A000036
:100170000000000100000000002C76D888DC674FEA
:100180000823DFC1DFAE59E1B1B796E5E3E453C61A
:100190003AE651997696E8E6C28426EB898C9B6212
:1001A000ED407C6FFCEFBC9C9F40F2BAA56FA5F4BC
:1001B00090055A2AF75C936B6CF9676DC11BFCE0E4
:1001C000E40D47FEF520E6B500D0ED902E03009437
:1001D0003577050080841E080000204E0A000000CC
:1001E000C80C333333330F986E12831141EF8D21D6
:1001F00014893BE65516CFFEE6DB18D1844B381B3D
:10020000F77C1D901DA4BBE424203284725E228101
:1002100000C9F124ECA1E53D2700002100240027BE
:10022000002A002D00300033000101000004010706
:10023000010A0100002200250028002B002E0031B9
:1002400000340002010000050108010B010000203C
:10025000002300260029002C002F0032000001009E
:100260000003010601090105050505070508080841
:1002700008020202020A0A08080404040401010137
:10028000010101010103030303030303030407073F
:10029000070C0C0C0C0C0C0C0C02020202060606DD
:1002A00006060606060B0B0B0B0B0B0B0B010210C5
:1002B0002020080810204010204080020102010880
:1002C0000402010102040810204080804020100830
:1002D0000402018004020180402010080402010889
:1002E00004020101020408102040800102040810E9
:1002F00020408000000A0B02090C0D0E08070304C1
:1003000001000000000000000000000000000000EC
:1003100000000000000000000000000000000012CB
:1003200011100000000000000000000000000000AC
:10033000000000000000000000008B3D11241FBEE3
:10034000CFEFD1E2DEBFCDBF00E00CBF17E0A0E0F1
:10035000B2E0E4EBF5EA00E00BBF02C007900D92BB
:10036000A03CB107D9F72DE0A0ECB7E001C01D9289
:10037000A23CB207E1F711E0CEE9D1E000E006C00F
:1003800021970109802FFE010E94D851CD39D10754
:1003900080E00807A9F70E94FC3D0C94D85230CEAB
:1003A000883591050CF04BC085359105CCF4803330
:1003B00091054CF58D3291059CF48C319105BCF47E
:1003C000893191056CF48E30910564F48B30910580
:1003D0003CF4009729F097FD08C00297049728F491
:1003E00081E008950F970997D8F380E00895863249
:1003F00091053CF4843291059CF74F970397A8F739
:10040000EFCF8997FBCF843491056CF4813491054B
:100410003CF78A3391052CF4873391050CF7C39789
:10042000EDCFCD97EBCF8E34910534F48B3491051D
:10043000BCF687549109E2CF81559109DFCF863808
:1004400091051CF5833891055CF68237910584F49B
:100450008F3691052CF6883691053CF4853691054A
:100460000CF0BECF8B559109C9CF89569109C6CFE3
:100470008C3791053CF4893791050CF0B1CF835747
:100480009109BCCF8D579109B9CF803D91058CF46E
:100490008D3C91050CF0A4CF843991053CF4813951
:1004A00091050CF09DCF8D589109A8CF895C9109D9
:1004B000A5CF8A3D91053CF4873D91050CF090CF86
:1004C000835D91099BCF8D5D910998CF9C01803E02
:1004D000910508F021C5FC018827EE58FD4F8F4F8C
:1004E0000C94D85152035F03680371037E038703A2
:1004F0008C078C078C078C078C079403A103AE0331
:100500008C07BB03C403CD03DA03E303EC03F50359
:10051000FE0307048C071004190422048C078C07BF
:100520008C072B0434043D048C078C0746045304C9
:100530008C078C078C0760046D047A048C07870491
:10054000900499048C078C078C07A204AB04B404B4
:100550008C07C104CE04DB048C078C078C07E804ED
:10056000F50402058C070F051C0529058C078C076F
:100570008C073605430550058C075D0566056F053C
:100580008C078C078C079305A005AD058C07BA0571
:10059000C705D4058C078C078C07E105EA05F30530
:1005A0008C078C078C078C078C078C078C07FC0545
:1005B00005060E068C071706200629068C078C07F1
:1005C0008C0732063F064C068C07590666067306F2
:1005D0008C078C078C0780068D069A068C07A70669
:1005E000B006B9068C078C078C07C206CB06D4066A
:1005F0008C078C078C078C078C078C078C078C0763
:100600008C078C078C07780581058A058C078C0779
:100610008C078C078C078C078C078C078C078C0742
:100620008C078C078C078C078C078C078C078C0732
:100630008C078C078C078C078C078C078C078C0722
:100640008C078C078C078C078C078C078C078C0712
:100650008C078C078C078C078C078C078C078C0702
:100660008C078C078C078C078C078C078C078C07F2
:100670008C078C078C07DD06E606F3068C0700075F
:10068000090716078C078C078C0723072C073907E7
:100690008C0746074F075C078C078C078C07690798
:1006A00072077F0781E090E0A0E0B0E08093F60859
:1006B0009093F708A093F808B093F9080895109262
:1006C000FA081092FB081092FC081092FD08089599
:1006D0001092FE081092FF08109200091092010972
:1006E000089581E090E0A0E0B0E08093020990934B
:1006F0000309A0930409B09305090895109206090F
:10070000109207091092080910920909089583E0D0
:1007100090E0A0E0B0E080930A0990930B09A093C9
:100720000C09B0930D09089588E790E0A0E0B0E0CF
:100730008093220990932309A0932409B09325095B
:10074000089588E790E0A0E0B0E0809326099093B8
:100750002709A0932809B0932909089588E790E014
:10076000A0E0B0E080932A0990932B09A0932C0974
:10077000B0932D0908951092320910923309109206
:1007800034091092350908951092360910923709EC
:100790001092380910923909089581E090E0A0E0A4
:1007A000B0E080933A0990933B09A0933C09B09341
:1007B0003D09089510923E0910923F091092400998
:1007C0001092410908951092420910924309109223
:1007D000440910924509089510924609109247095C
:1007E0001092480910924909089510924A091092EE
:1007F0004B0910924C0910924D09089510924E0920
:1008000010924F09109250091092510908951092B8
:1008100052091092530910925409109255090895E3
:1008200010925A0910925B0910925C0910925D09AE
:10083000089510925E0910925F091092600910925B
:100840006109089510926209109263091092640977
:10085000109265090895109272091092730910920E
:10086000740910927509089510927609109277090B
:100870001092780910927909089510927A091092CD
:100880007B0910927C0910927D09089581E090E027
:10089000A0E0B0E08093860990938709A09388092F
:1008A000B0938909089581E090E0A0E0B0E08093E2
:1008B0008A0990938B09A0938C09B0938D090895B0
:1008C0008CE291E0A0E0B0E080939A0990939B09BC
:1008D000A0939C09B0939D0908958CE291E0A0E05B
:1008E000B0E080939E0990939F09A093A009B093D4
:1008F000A10908958CE291E0A0E0B0E08093A20904
:100900009093A309A093A409B093A5090895109208
:10091000AA091092AB091092AC091092AD09089582
:100920001092AE091092AF091092B0091092B1095D
:1009300008951092B2091092B3091092B40910925E
:10094000B50908951092C2091092C3091092C40902
:100950001092C50908951092C6091092C709109205
:10096000C8091092C909089581E090E0A0E0B0E0C4
:100970008093CA099093CB09A093CC09B093CD0979
:10098000089585E090E0A0E0B0E08093D2099093D4
:10099000D309A093D409B093D509089585E090E0D8
:1009A000A0E0B0E08093D6099093D709A093D8092E
:1009B000B093D909089589E190E0A0E0B0E0809378
:1009C000DA099093DB09A093DC09B093DD0908955F
:1009D00082E390E0A0E0B0E08093EA099093EB0915
:1009E000A093EC09B093ED09089582E390E0A0E0B4
:1009F000B0E08093EE099093EF09A093F009B093D3
:100A0000F109089582E390E0A0E0B0E08093F2095C
:100A10009093F309A093F409B093F509089582E344
:100A200090E0A0E0B0E08093FA099093FB09A093D6
:100A3000FC09B093FD09089582E390E0A0E0B0E0E6
:100A40008093FE099093FF09A093000AB093010AD6
:100A5000089582E390E0A0E0B0E08093020A9093D2
:100A6000030AA093040AB093050A089580E991E06F
:100A7000A0E0B0E08093120A9093130AA093140AA6
:100A8000B093150A089580E991E0A0E0B0E080936A
:100A9000160A9093170AA093180AB093190A08959A
:100AA00080E991E0A0E0B0E080931A0A90931B0ADD
:100AB000A0931C0AB0931D0A08951092220A109266
:100AC000230A1092240A1092250A08951092260AE9
:100AD0001092270A1092280A1092290A089510925B
:100AE0002A0A10922B0A10922C0A10922D0A0895AD
:100AF00010923A0B10923B0B10923C0B10923D0B54
:100B0000089510923E0B10923F0B1092400B1092E2
:100B1000410B08951092420B1092430B1092440B1C
:100B20001092450B089588E592E0A0E0B0E0809334
:100B30003A0A90933B0AA0933C0AB0933D0A089569
:100B400088E592E0A0E0B0E080933E0A90933F0AEF
:100B5000A093400AB093410A089588E592E0A0E08E
:100B6000B0E08093420A9093430AA093440AB09362
:100B7000450A08958EE190E0A0E0B0E080934A0A33
:100B800090934B0AA0934C0AB0934D0A08958EE1BE
:100B900090E0A0E0B0E080934E0A90934F0AA093BB
:100BA000500AB093510A08958EE190E0A0E0B0E0C1
:100BB0008093520A9093530AA093540AB093550A13
:100BC00008951092620A1092630A1092640A1092B9
:100BD000650A08951092660A1092670A1092680AD0
:100BE0001092690A089510926A0A10926B0A109284
:100BF0006C0A10926D0A089510928A0A10928B0A5C
:100C000010928C0A10928D0A089510928E0A1092FA
:100C10008F0A1092900A1092910A08951092920AE7
:100C20001092930A1092940A1092950A08951092C5
:100C30009A0A10929B0A10929C0A10929D0A08959B
:100C400010929E0A10929F0A1092A00A1092A10A76
:100C500008951092A20A1092A30A1092A40A109268
:100C6000A50A089585E090E0A0E0B0E08093B20A84
:100C70009093B30AA093B40AB093B50A089585E09F
:100C800090E0A0E0B0E08093B60A9093B70AA093FA
:100C9000B80AB093B90A089585E090E0A0E0B0E00A
:100CA0008093BA0A9093BB0AA093BC0AB093BD0A82
:100CB000089584EB95E1A0E0B0E08093C20A9093A0
:100CC000C30AA093C40AB093C50A089584EB95E1C2
:100CD000A0E0B0E08093C60A9093C70AA093C80A28
:100CE000B093C90A089584EB95E1A0E0B0E0809349
:100CF000CA0A9093CB0AA093CC0AB093CD0A089568
:100D000085E090E0A0E0B0E08093DA0A9093DB0AFF
:100D1000A093DC0AB093DD0A089585E090E0A0E09E
:100D2000B0E08093DE0A9093DF0AA093E00AB093CC
:100D3000E10A089585E090E0A0E0B0E08093E20A47
:100D40009093E30AA093E40AB093E50A0895109201
:100D5000EA0A1092EB0A1092EC0A1092ED0A08953A
:100D60001092EE0A1092EF0A1092F00A1092F10A15
:100D700008951092F20A1092F30A1092F40A109257
:100D8000F50A08951092020B1092030B1092040BB7
:100D90001092050B08951092060B1092070B1092FB
:100DA000080B1092090B089510920A0B10920B0B6E
:100DB00010920C0B10920D0B089510921A0C1092B9
:100DC0001B0C10921C0C10921D0C08958CE390E0EB
:100DD000A0E0B0E080931E0C90931F0CA093200C19
:100DE000B093210C089581E090E0A0E0B0E0809302
:100DF000220C9093230CA093240CB093250C0895FF
:100E000010922A0C10922B0C10922C0C10922D0C7C
:100E100008958CE390E0A0E0B0E080932E0C9093D6
:100E20002F0CA093300CB093310C089581E090E02A
:100E3000A0E0B0E08093320C9093330CA093340C7C
:100E4000B093350C08951092420C1092430C1092FE
:100E5000440C1092450C08958CE390E0A0E0B0E0C3
:100E60008093460C9093470CA093480CB093490C88
:100E7000089581E090E0A0E0B0E080934A0C909368
:100E80004B0CA0934C0CB0934D0C08951092520C47
:100E90001092530C1092540C1092550C08958CE340
:100EA00090E0A0E0B0E08093560C9093570CA09394
:100EB000580CB093590C089581E090E0A0E0B0E0A8
:100EC00080935A0C90935B0CA0935C0CB0935D0CD8
:100ED000089510926A0C10926B0C10926C0C109288
:100EE0006D0C08958CE390E0A0E0B0E080936E0C70
:100EF00090936F0CA093700CB093710C089581E0E7
:100F000090E0A0E0B0E08093720C9093730CA093FB
:100F1000740CB093750C0895220F331F220F331FEA
:100F2000F901EA50F74F108211821282138208955C
:100F3000AF92BF92CF92DF92EF92FF920F931F93E7
:100F4000CF93DF936C017B018B01040F151FEB0125
:100F50005E01AE18BF08C017D10759F06991D601DC
:100F6000ED91FC910190F081E02DC6011995892B3E
:100F700079F7C501DF91CF911F910F91FF90EF900D
:100F8000DF90CF90BF90AF900895FC01538D448DBA
:100F9000252F30E0842F90E0821B930B541710F024
:100FA000CF96089501970895FC01918D828D981731
:100FB00061F0A28DAE0FBF2FB11D5D968C91928D09
:100FC0009F5F9F73928F90E008958FEF9FEF08953A
:100FD000FC01918D828D981731F0828DE80FF11D03
:100FE000858D90E008958FEF9FEF0895FC01918D1E
:100FF000228D892F90E0805C9F4F821B91098F7317
:10100000992708958EE79CE0F1DF21E0892B09F410
:1010100020E0822F0895FC01A48DA80FB92FB11DE7
:10102000A35ABF4F2C91848D90E001968F7399271E
:10103000848FA689B7892C93A089B1898C918370FC
:1010400080648C93938D848D981306C00288F389F5
:10105000E02D80818F7D80830895EF92FF920F9322
:101060001F93CF93DF93EC0181E0888F9B8D8C8D54
:1010700098131AC0E889F989808185FF15C09FB748
:10108000F894EE89FF896083E889F989808183700B
:10109000806480839FBF81E090E0DF91CF911F91BA
:1010A0000F91FF90EF900895F62E0B8D10E00F5FDB
:1010B0001F4F0F731127E02E8C8D8E110BC00FB6B2
:1010C00007FCFACFE889F989808185FFF5CFCE0149
:1010D000A2DFF2CFEB8DEC0FFD2FF11DE35AFF4F96
:1010E000F0829FB7F8940B8FEA89FB898081806238
:1010F000D0CF682F8EE79CE0B0CFCF93DF93EC0189
:10110000888D8823B1F0AA89BB89E889F9898C91F7
:1011100085FD03C0808186FD0CC00FB607FCF7CFAC
:101120008C9185FFF2CF808185FFEDCFCE0173DFFB
:10113000EACFDF91CF91089580E090E0892B21F0F4
:1011400061DF81110E94000080E090E0892B49F06E
:1011500080E090E0892B29F00E94000081110E941C
:10116000000080E090E0892B49F080E090E0892B3E
:1011700029F00E94000081110E94000080E090E0B0
:10118000892B49F080E090E0892B29F00E94000033
:1011900081110C94000008958150823108F05AC0EA
:1011A000E82FF0E08827E852F74F8F4F0C94D85182
:1011B000F808FC08EA08F008F4082A09FF080509FD
:1011C00009090F09130917091D0921092A09250908
:1011D0002B092F09809180008F77809380000895DC
:1011E000809180008F7DF9CF80918000877FF5CF3F
:1011F00084B58F7784BD089584B58F7DFBCF8091B2
:10120000B0008F778093B00008958091B0008F7DFB
:10121000F9CF809190008F7780939000089580910E
:1012200090008F7DF9CF80919000877FF5CF8091DE
:10123000A0008F778093A00008958091A0008F7DFB
:10124000F9CF8091A000877FF5CF809120018F7723
:10125000809320010895809120018F7DF9CF8091A6
:101260002001877FF5CFCF93DF93282F30E0F9015E
:10127000ED50FD4F8491F901E355FD4FD491F901F3
:10128000E959FD4FC491CC2399F0811185DFEC2FF2
:10129000F0E0EE0FFF1FE35BFD4FA591B491EC91E1
:1012A000ED2381E090E009F480E0DF91CF91089593
:1012B00080E090E0FACF1F93CF93DF93282F30E0A8
:1012C000F901ED50FD4F8491F901E355FD4FD491A3
:1012D000F901E959FD4FC491CC23A1F0162F8111DA
:1012E0005BDFEC2FF0E0EE0FFF1FED5CFD4FA591F3
:1012F000B4918FB7F894EC91111108C0D095DE230A
:10130000DC938FBFDF91CF911F910895DE2BF8CF33
:10131000CF93DF9390E0FC01E355FD4F2491895971
:101320009D4FFC0184918823C9F090E0880F991F9C
:10133000FC01E75EFD4FA591B491FC01ED5CFD4F12
:10134000C591D49161110DC09FB7F8948C912095EF
:1013500082238C938881282328839FBFDF91CF919C
:101360000895623051F49FB7F8943C91822F809594
:1013700083238C93E8812E2BEFCF8FB7F894EC91D9
:101380002E2B2C938FBFEACF8230910538F0880F37
:10139000991F880F991F05970197F1F708953FB797
:1013A000F8948091D6079091D707A091D807B09173
:1013B000D90726B5A89B05C02F3F19F00196A11D9E
:1013C000B11D3FBFBA2FA92F982F8827BC01CD018F
:1013D000620F711D811D911D42E0660F771F881FEE
:1013E000991F4A95D1F708958F929F92AF92BF921D
:1013F000CF92DF92EF92FF926B017C01D0DF4B0125
:101400005C01C114D104E104F104B1F0C8DF681932
:1014100079098A099B09683E73408105910588F323
:1014200021E0C21AD108E108F10888EE880E83E0B5
:10143000981EA11CB11CE5CFFF90EF90DF90CF90DC
:10144000BF90AF909F908F9008952FB7F8946091C0
:10145000D2077091D3078091D4079091D5072FBF01
:101460000895CF92DF92EF92FF92CF93DF93EC013A
:10147000603282E07807CCF5653B710514F064EBCF
:1014800070E0898128E830E0281B310987FD339519
:10149000220F331F220F331F6901330FEE08FF089D
:1014A0008A8128E532E0281B310987FD3395220F18
:1014B000331F220F331F032E000C440B550B2C1926
:1014C0003D094E095F09DB0177FF02C0B0E0A0E0F3
:1014D0000E94805024EB30E040E050E00E945A50DF
:1014E000C20ED31EE41EF51EB601E881E03370F58E
:1014F000298188E890E0821B910927FD9395880F48
:10150000991F880F991F681779077CF02A8188E551
:1015100092E0821B910927FD9395880F991F880FF0
:10152000991F681779070CF4CB010297880F991F50
:101530004FB7F8942E2F30E0F901EE0FFF1FE20FA6
:10154000F31FE55EF24F928381834FBFDF91CF910E
:10155000FF90EF90DF90CF9008951F93CF93DF938C
:10156000EC01162F8881803308F04DC061E0812F97
:10157000CFDE8881282F30E0F901EE0FFF1FE20F48
:10158000F31FE55EF24F1F736081607C612B608307
:1015900019821A822CE0622F0E94CC51829FB001E6
:1015A000112430E020E0AB01420F531FFA01EE0F8F
:1015B000FF1FE40FF51FE55EF24F908196FD16C008
:1015C0002F5F3F4F2C30310571F7813009F51092B4
:1015D000800082E080938100109285001092840048
:1015E000B19A80916F00826080936F00E8818E2FA6
:1015F00090E0FC01EE0FFF1FE80FF91FE55EF24FD0
:101600008081806480838881DF91CF911F910895CC
:10161000823061F4109290008093910010929500B6
:101620001092940088BB80937100E0CF833069F4FE
:101630001092A00082E08093A1001092A500109269
:10164000A40089BB80937200D1CF8111CFCF1092BB
:10165000200182E080932101109225011092240143
:101660008ABB80937300C2CFAF92BF92CF92DF92BA
:10167000EF92FF920F931F93CF93DF936B017A0149
:10168000EC01C353D84F28813CE0389F8001399F3B
:10169000100D1124A090AB0DB12C27FF1FC0FB0132
:1016A0001182108288818F5F888388819801280F3A
:1016B000311D87FD3A95F6012A153B051CF48881FA
:1016C0008C30BCF180819181049680349C4908F46F
:1016D00071C0F6018081918104966EC08881980165
:1016E000280F311D87FD3A952A153B05DCF68881C8
:1016F000A801480F511D87FD5A95FA01EE0FFF1FF3
:10170000E40FF51FE55EF24F808186FFCBCF888125
:10171000F801E80FF11D87FDFA95CF01EE0FFF1FCD
:10172000E80FF91FE55EF24F808160E08F73C3DD43
:10173000B9CF808191812881A801420F511D27FDD9
:101740005A959A01FA01EE0FFF1FE20FF31FE55EB3
:10175000F24F21813281820F931FF70191838083A1
:1017600088819801280F311D87FD3A95F901EE0F08
:10177000FF1FE20FF31FE55EF24F808186FF21C05D
:101780008881080F111D87FD1A95F801EE0FFF1FC4
:10179000E00FF11FE55EF24F808161E08F73DF9112
:1017A000CF911F910F91FF90EF90DF90CF90BF905E
:1017B000AF9081CD80E49CE9F701918380838FEF26
:1017C0008883DF91CF911F910F91FF90EF90DF9071
:1017D000CF90BF90AF90089508950895089508950B
:1017E0000895EBE0F1E08081877F80830895EBE04E
:1017F000F1E080818860808308958E9808958E9AA4
:10180000089514980895149A089588980895889AC8
:10181000089560E0FC0183854ECD60E0FC01858188
:101820004ACD61E0FC01838546CD61E0FC01858104
:1018300042CDCF93DF93EC01FC01E359FF4F1082BF
:10184000379781E0808360E08D8135DD8F859889D1
:10185000892B29F060E08B85DF91CF912CCDDF9132
:10186000CF910895CF93DF93EC018B89FCDC2E8917
:101870002817190621F48F89DF91CF91089580E010
:10188000FBCFCF93DF93EC018989EDDC2E892817FC
:10189000190621F48F89DF91CF91089580E0FBCF65
:1018A000CF93DF93EC018F819DA561E0911101C081
:1018B00060E001DD8D859EA5992321F09FA561E063
:1018C000911101C060E0DF91CF91F5CCCF93DF9310
:1018D000EC018F819DA560E0911101C061E0EBDC1E
:1018E0008D859EA5992321F09FA560E0911101C0EF
:1018F00061E0DF91CF91DFCCCF93DF93EC0161E02A
:101900008985D9DC8EA5882319F061E08F85D3DC29
:10191000C559DF4F1882DF91CF910895CF93DF93A0
:10192000EC0160E08985C7DC8EA5882319F060E0B2
:101930008F85C1DCC559DF4F81E08883DF91CF916E
:101940000895CF92DF92EF92FF920F931F93CF9360
:10195000DF93FC0142AF53AF64AF75AFDC01DE969D
:101960004D935D936D937C93139714960D931D93F4
:101970002D933C931397EC01CA5BDF4FE88284A957
:10198000882351F094A591114CC037FF50C01D928F
:101990001D921D921C92139745A956A967A970AD77
:1019A00014161506160617063CF591AD992321F17C
:1019B0000D911D912D913C9113976801790137FF8D
:1019C00007C0CC24DD247601C01AD10AE20AF30A4A
:1019D0004C155D056E057F057CF437FF07C07095DB
:1019E0006095509541955F4F6F4F7F4F4D935D933D
:1019F0006D937C931397892FDF01AD5ABF4F1D92D2
:101A00001D921D921C921397ED59FF4F91E0908308
:101A1000DF91CF911F910F91FF90EF90DF90CF90CA
:101A2000089510161106120613060CF4B0CF80E0CC
:101A3000B3CF0F931F93CF93DF93EC01062F8D89C4
:101A400081110DC0CE011DDF182FCE010BDF01115A
:101A5000182F812FDF91CF911F910F910895CE0103
:101A600001DF182FCE010DDFF2CFCF93DF93EC0112
:101A7000FC01E359FF4F81E08083AE01425C5F4F80
:101A8000FA0180819181A281B3819E012C593F4F3F
:101A9000F9012081222309F440C00196A11DB11D46
:101AA000FA0180839183A283B383FE01E059FF4F43
:101AB00020813181C901959587958C0F9D1F3297A3
:101AC0000190F081E02D20FF08C0DC012D913C91B8
:101AD000E20FF31F0190F081E02D19958F85988911
:101AE000892BF9F0FE01EC58FF4F20813181C901AB
:101AF000959587958C0F9D1FCE58DF4FE881F98112
:101B000020FF08C0DC012D913C91E20FF31F0190F2
:101B1000F081E02DDF91CF9119940197A109B109CE
:101B2000BFCFDF91CF9108958F929F92AF92BF92D6
:101B3000CF92DF92EF92FF920F931F93CF93DF9399
:101B4000EC01FC01ED5AFF4F60817181828193812C
:101B50000E942C4F6B017C0168A979A98AA99BA9D5
:101B60000E942E4F9B01AC0160E074E284E799E48F
:101B70000E941C514B015C01FE01E15AFF4F608144
:101B80007181828193810E942C4F9B01AC01C50120
:101B9000B4010E941C514B015C018E01095A1F4F78
:101BA00020E030E040E05FE30E948D4FA701960106
:101BB0000E94B8500E948951F8016083718382832A
:101BC0009383C55ADF4FA5019401C701B6010E9456
:101BD000B8500E948951688379838A839B83DF91FF
:101BE000CF911F910F91FF90EF90DF90CF90BF901A
:101BF000AF909F908F9008950F931F93CF93DF9393
:101C0000FC01E359FF4F20812223B9F07A9700812C
:101C100011812281338138964081518162817381A3
:101C2000041715072607370710F1EC0102DECE0175
:101C3000DF91CF911F910F9177CFFC01ED59FF4FAD
:101C400020812223A1F070970081118122813381AC
:101C500034964081518162817381041715072607EC
:101C6000370728F0DF91CF911F910F91FECEDF91C2
:101C7000CF911F910F910895FC01ED59FF4F2081E5
:101C8000222361F0709780819181A281B3810196B6
:101C9000A11DB11D80839183A283B38308950F9307
:101CA0001F93FC01EA5BFF4F2081211112C038977E
:101CB000008111812281338134964081518162817A
:101CC000738104171507260737073CF41F910F91FE
:101CD000FDCDFC0124A52111F9CF1F910F91E0CD7D
:101CE000FC011382128214828CE291E0A0E0B0E049
:101CF000808F918FA28FB38F42E350E060E070E05D
:101D0000448F558F668F778F40A351A362A373A32F
:101D100084A395A3A6A3B7A388E790E0A0E0B0E0D2
:101D200080A791A7A2A7B3A714A615A616A617A6C3
:101D300084E690E0A0E0B0E080AB91ABA2ABB3ABA7
:101D400014AA15AA16AA17AA10AE11AE12AE13AE97
:101D500014AE15AEDF01DE961D921D921D921C92EF
:101D6000139714961D921D921D921C921397149610
:101D70001C9211961D921D921D921C9213971496FF
:101D80001D921D921D921C92139714961D921D92E6
:101D90001D921C92139714961D921D921D921C92D7
:101DA000139714961D921D921D921C9213971496D0
:101DB0001D921D921D921C92139714961D921D92B6
:101DC0001D921C92139714961C9211961C921196B8
:101DD0001C9211961C9211961C9211961C921196AF
:101DE0001C9211961C9211961C9211961C9211969F
:101DF0001C9216821582108617821286118614860E
:101E0000138616861586108A1786128A118A148AF6
:101E1000138A119685E19CE011969C938E931296FD
:101E200011961C921E92129681E19CE011969C9351
:101E30008E93129611961C921E9212968DE09CE043
:101E400011969C938E93129611961C921E92129646
:101E500089E09CE08D939C93E458FF4F118210829F
:101E600008950895089508958FEF9FEF08950895B8
:101E70000895CF93DF93EC018881F5D921E0892B78
:101E800009F420E02C878C81EED921E0892B09F41C
:101E900020E02E878C8D9D8D0197D1F48A81E3D926
:101EA00021E0892B09F420E02D878E81DCD921E007
:101EB000892B09F420E02F879C858D85981729F0C0
:101EC0008E85281711F09A878B87DF91CF9108951F
:101ED0008C858A872B87F9CF0F93FC019285908799
:101EE00083858187A48DB58D119721F4621721F028
:101EF000401711F0628743878385882381F08285AC
:101F000091110FC0882359F080899189A289B389E2
:101F10000197A109B109808B918BA28BB38B0F9193
:101F200008958111FCCF80899189A289B389019696
:101F3000A11DB11DF0CF4F925F926F927F928F9251
:101F40009F92AF92BF92CF92DF92EF92FF92CF9388
:101F5000DF93EC016C897D898E899F8988889988B7
:101F6000AA88BB88CE8CDF8C0D2C000CEE08FF08F5
:101F7000603127E272078105910529F016161706D0
:101F800018061906ACF0A7019601C501B4010E941C
:101F9000BD51DF91CF91FF90EF90DF90CF90BF9038
:101FA000AF909F908F907F906F905F904F9008952B
:101FB0000E942E4F20E030E44CE156E40E941C5178
:101FC0002B013C01488E598E6A8E7B8EC501B4016F
:101FD0000E942E4FA30192010E948D4F4B015C0184
:101FE000C701B6010E942E4F9B01AC01C501B4018F
:101FF0000E948D4F0E948451CCCFFC01118210822F
:10200000138212821582148217821682108611861C
:10201000128613861486158616861786108A118AEC
:10202000128A138A108E118E128E138E158E148EB4
:10203000178E168E10A211A212A213A214A215A21C
:1020400016A217A210A611A612A613A614A615A6CC
:1020500081E090E097A786A780E197E2A0E0B0E05A
:10206000848B958BA68BB78B08950895089508955A
:10207000089508950F931F93CF93DF938B01EA0187
:10208000AB01415051094433510508F0E9C02230F9
:10209000310508F0E5C048E3429FF001439FF00D91
:1020A0001124E80FF91FE60FF71F81E080836C2FE2
:1020B000232B09F4D2C061E0802F2AD9209749F45C
:1020C00060E0802FF8D8CE01DF91CF911F910F9162
:1020D0000895CF3FD10511F461E0BFC0F801ED5084
:1020E000FD4FE491E150E23108F0B2C0F0E0882702
:1020F000E358FF4E8F4F0C94D8518F1096109B10C1
:10210000A510AF102811B910C110C910D310DD10DF
:10211000E710F610001128110A1114111E1184B5D0
:10212000806884BDC7BDD0E0C0E0CDCF84B58062FB
:1021300084BDC8BDF8CF8091800080688093800006
:10214000D0938900C0938800EECF80918000806298
:1021500080938000D0938B00C0938A00E4CF80915D
:102160008000886080938000D0938D00C0938C00A5
:10217000DACF8091B00080688093B000C093B30044
:10218000D2CF8091B00080628093B000C093B40041
:10219000CACF80919000806880939000D09399007E
:1021A000C0939800C0CF809190008062809390008F
:1021B000D0939B00C0939A00B6CF80919000886026
:1021C00080939000D0939D00C0939C00ACCF8091F1
:1021D000A00080688093A0008091A0008F7B8093F6
:1021E000A000D093A900C093A8009DCF8091A0002B
:1021F00080628093A000D093AB00C093AA0093CFDD
:102200008091A00088608093A000D093AD00C0931F
:10221000AC0089CF80912001806880932001D09309
:102220002901C09328017FCF809120018062809393
:102230002001D0932B01C0932A0175CF80912001FA
:10224000886080932001D0932D01C0932C016BCF27
:1022500060E0C038D1050CF03FCF802F2CD863CF81
:10226000C1E0D0E030CF0895CF93DF93D0E0C0E05D
:10227000CE010E94D001882319F0CE010E9466028F
:102280002196C13ED105A1F7DF91CF910895089520
:102290002F923F924F925F926F927F928F929F9276
:1022A000AF92BF92CF92DF92EF92FF920F931F9364
:1022B000CF93DF9300D01F92CDB7DEB79C838B8383
:1022C0004B015A011901FA82E982FA0140805180DA
:1022D0006280738020E030E0A901C301B2010E9456
:1022E000B551181674F4F601208131814281538171
:1022F000C301B2010E94B750F501608371838283EC
:102300009383F8014080518062807380F401A68D30
:10231000B78D20893189428953890E9480506B0191
:102320007C01EB81FC81EC59FF4F8081882309F40B
:102330003FC0C414D504E604F7040CF43EC0F80111
:10234000C082D182E282F3828B819C81CE969C8373
:102350008B83FC0180819181A281B381F101808313
:102360009183A283B383E981FA8180819181892B52
:1023700041F0C401E0DDEB81FC81608371838283E5
:1023800093830F900F900F900F90DF91CF911F913B
:102390000F91FF90EF90DF90CF90BF90AF909F9004
:1023A0008F907F906F905F904F903F902F90089507
:1023B0004C145D046E047F0414F6F50140805180D6
:1023C0006280738020E030E04AEF56E4C301B2013E
:1023D0000E94284F87FFB3CF20E030E040E85FE362
:1023E000C301B2010E94B850F501608371838283FA
:1023F0009383A5CFCF93DF93EC01FC01E05FFC4F0B
:102400001082EE58F1098081811103C0CE014096FF
:1024100073DAFE01ED57FD4F8081811104C0CE01BA
:1024200082579F4F69DAFE01EC57FD4F8081811181
:1024300004C0CE01845F9E4F5FDA64E670E080E006
:1024400090E0DF91CF910C94F409089508950895D8
:10245000089508958091CB079091CC07892B09F0BE
:1024600040C08FE090E00E94AF49FC0181E090E025
:10247000A0E0B0E080839183A283B38384839583BB
:10248000A683B78380879187A287B3871586148632
:1024900016861092DC081092DD081092DE08109269
:1024A000DF081092E0081092E1081092E208109202
:1024B000E3081092E4081092E5081092E6081092E2
:1024C000E70810927A0C10927B0C10927C0C109200
:1024D0007D0C10920C0810920B08F093CC07E0933F
:1024E000CB078091CB079091CC070895B3DF83E0B1
:1024F0000E94330921E0892B09F420E02093F008A1
:10250000A9DF82E00E94330921E0892B09F420E051
:102510002093F1089FDF8EE00E94330921E0892B90
:1025200009F420E02093F20895DF8FE00E94330940
:1025300021E0892B09F420E02093F3088BDF82E16E
:102540000E94330921E0892B09F420E02093F4084C
:1025500081DF83E10E94330921E0892B09F420E027
:102560002093F508089576DFC1CF74DFFC0116864D
:1025700090E080E008958091C7079091C807892B6B
:1025800041F481E090E00E94AF499093C8078093A6
:10259000C7078091C7079091C80708950F931F93AD
:1025A000CF93DF938B01E7DFF801C2A1D3A1868D22
:1025B000978D8530910529F14CF40497B1F090E0A6
:1025C00080E0DF91CF911F910F91089586309105A2
:1025D00011F10B97A1F76BE070E085EB9DE00E9495
:1025E000AD0ABE0185EB9DE009C064E070E08CEAB5
:1025F0009DE00E94AD0ABE018CEA9DE00E94310A76
:10260000DECF65E070E08FEA9DE00E94AD0ABE017A
:102610008FEA9DE0F3CF66E070E082EB9DE00E94E0
:10262000AD0ABE0182EB9DE0E9CF8091C407909195
:10263000C507892B91F480E790E00E94AF49FC0127
:1026400031969C012B5C3F4F119217AAE217F307BA
:10265000D9F79093C5078093C4078091C4079091E0
:10266000C5070895CF93DF93EB01DFDF6AA98E8D55
:102670000E94880990E080E0DF91CF9108954F9209
:102680005F926F927F92AF92BF92CF92DF92EF9262
:10269000FF920F931F93CF93DF93EB01C6DF8C0163
:1026A000CAA8DBA84EA45FA468A879A8AEA0BFA062
:1026B000EE8CFF8C4AA15BA19601B701DBDCC30164
:1026C000B2010E94F4099601A501B701C801D2DC4C
:1026D00090E080E0DF91CF911F910F91FF90EF90FC
:1026E000DF90CF90BF90AF907F906F905F904F90B2
:1026F0000895CF93DF93EB0198DF2AA93BA94AA164
:102700005BA16E8D7F8DB6DC90E080E0DF91CF9194
:102710000895FC0101900020E9F73197AF01481BB3
:10272000590BBC018EE79CE00C9498078F929F9206
:10273000AF92BF920F931F93CF93DF93CDB7DEB7C6
:10274000A1970FB6F894DEBF0FBECDBF19A24230DD
:1027500008F44AE08E010F5D1F4F842E912CB12C9E
:10276000A12CA50194010E948650E62FB901CA014F
:10277000EA30ECF4E05DD801EE938D01232B242B9D
:10278000252B79F790E080E0109711F0CD01C1DFA3
:10279000A1960FB6F894DEBF0FBECDBFDF91CF91EB
:1027A0001F910F91BF90AF909F908F900895E95C1B
:1027B000E2CFAFCF882319F088E197E0FACF81E12B
:1027C00097E0FCCFCF92DF92EF92FF92CF93DF930F
:1027D00097FF18C06B017C018DE20E947908EC0123
:1027E00066277727CB016C197D098E099F094AE07E
:1027F0009DDF8C0F9D1FDF91CF91FF90EF90DF90B9
:10280000CF9008954AE0DF91CF91FF90EF90DF9055
:10281000CF908CCFBC01990F880B990BD3CF88E850
:1028200093E0C7DF60917A0C70917B0C80917C0CF7
:1028300090917D0CC7DF8CE897E0BBCF0F931F937F
:10284000CF93DF938C01EB018AE693E0B2DF87EB55
:1028500093E0AFDFF80180810E947908CE01DADFD2
:10286000F9DDDF91CF911F910F91D9CFEF92FF92B8
:102870000F931F93CF93DF93182F092F7B016115BF
:10288000710569F50E94330931E020E0019709F0F4
:1028900030E0C32FD22F82E0E816F10408F045C0E3
:1028A0008BE893E086DF87EB93E083DF8FE893E0AC
:1028B00080DF812F902FAEDF87EB93E07ADF8DEB07
:1028C00097E077DFCE01A6DFC5DDA9DF90E080E0ED
:1028D000DF91CF911F910F91FF90EF900895D0E07D
:1028E000C0E061307105B9F6812F163310F08AEC23
:1028F000810F20917B00982F9870277F922B9093C7
:102900007B008770806480937C0080917A00806473
:1029100080937A0080917A0086FDFCCF80917800C8
:10292000C0917900DC2FC82FB6CF81E090E0D0CFE6
:102930000F931F93CF93DF93FC01208131812115E9
:102940003105C1F1EC01822F0E94330921E0892B6E
:1029500009F420E02B876A85261701F11E821F8269
:10296000188619860E811F81288539858A819B8169
:10297000AC81BD81081719072A073B07DCF081E00D
:10298000682788810E945B0950DE70E060E08881E2
:102990009981DF91CF911F910F9168CF8E819F8197
:1029A000A885B9850196A11DB11D8E839F83A88737
:1029B000B987D8CFDF91CF911F910F910895CF9311
:1029C000DF93EB0132DE6AA97BA98E8D9F8D4EDFEE
:1029D00090E080E0DF91CF910895CF93DF9381E97C
:1029E00093E0E7DE85E993E0E4DEC0EFD8E088819C
:1029F000E1DE89E993E0DDDE8981DCDE8DE993E0CB
:102A0000D8DE8A81D7DE81EA93E0D3DE8B81D2DE05
:102A100085EA93E0CEDE8C81CDDE89EA93E0C9DEE3
:102A20008D81C8DEDF91CF91FACE14DDD6CF8DEA4D
:102A300093E0BFDE0FDD5ADD0DDDCFDFF6DD70E0A8
:102A400060E088E090E012DFF0DD70E060E089E0B7
:102A500090E00CDFEADD70E060E08AE090E006DF05
:102A6000E4DD70E060E08DE090E000DF90E080E089
:102A7000089584EB93E09DDE88E092E09ADEEADC44
:102A8000CEDE90E080E00895CF92DF92EF92FF9249
:102A9000CF93DF93EB01CB010E94D001882351F14A
:102AA000FE01EE0FFF1FEE0FFF1FEA50F74FC08031
:102AB000D180E280F38089EB93E07BDE87EB93E0CB
:102AC00078DE8FE893E075DECE01A4DE87EB93E03D
:102AD00070DE8DEB97E06DDEC701B60173DEBADC08
:102AE0009EDE90E080E0DF91CF91FF90EF90DF904D
:102AF000CF9008958DEB93E05CDEF3CF0F931F939F
:102B0000CF93DF938C01D0E0C0E0CE010E94D001D2
:102B1000882319F0BE01C801B7DF2196C13ED10557
:102B2000A1F7DF91CF911F910F9108952F923F92BE
:102B30004F925F926F927F928F929F92AF92BF92CD
:102B4000CF92DF92EF92FF920F931F93CF93DF9379
:102B5000CDB7DEB762970FB6F894DEBF0FBECDBF1C
:102B60008C01FC01FE9640815181628173811C01C0
:102B700022E4220E311CF10180819181A281B38176
:102B80007801F6E4EF0EF11CF701B08098012C59A2
:102B90003F4F49017F966F01BB2089F1F80124A5C1
:102BA000F401208321E0F6012083411551056105E0
:102BB000710559F4F801848C958CA68CB78CE15A78
:102BC000FF4F80829182A282B382F80142AC53AC63
:102BD00064AC75AC98012D593F4F59014816590600
:102BE0006A067B06A4F5481759076A077B07CCF1EC
:102BF000D7018C91811135C0D5011C9239C121E0DA
:102C0000481759076A077B070CF020E0F40120837E
:102C10002A013B0177FF07C0442455243201441A9E
:102C2000550A660A770A4C015D01B7FF07C0882480
:102C300099245401881A990AAA0ABB0A21E0481467
:102C400059046A047B040CF0AECF20E0ACCF8415AD
:102C50009505A605B70564F684179507A607B70777
:102C60003CF6F5018081882339F2D7018C918111DE
:102C70000EC0F70180818111BFCFD6016C9181E038
:102C80006827C8010E94190D8111B6CF06C060E007
:102C9000C8010E94190D8111ECCFD80194962D9195
:102CA0003D914D915C91979729833A834B835C8347
:102CB00058962D913D914D915C915B972D833E836C
:102CC0004F8358875C962D913D914D915C915F9714
:102CD00029873A874B875C87F10180819181A281A6
:102CE000B381F801FE96C080D180E280F380F801C4
:102CF00042AD53AD64AD75ADE959FF4F10823196C9
:102D000010823801F9E66F0E711CF30110829801F0
:102D100026593F4FF9011082329610824C015D0115
:102D2000841A950AA60AB70AB7FE08C0B094A09400
:102D300090948094811C911CA11CB11C48175907C8
:102D40006A077B072CF0C81AD90AEA0AFB0A04C0F2
:102D5000C41AD50AE60AF70AD501C401B595A795A4
:102D6000979587958D879E87AF87B88BD801A45993
:102D7000BF4F1D018C149D04AE04BF0408F09DC01C
:102D8000F80100A0F1A1E02DFA8BE98B81E0D901D7
:102D90008C93F1018083F8018481882309F45CC05D
:102DA0000E94250AD80112964D905C90052C000CCB
:102DB000660877086419750986099709693E7340A2
:102DC0008105910508F448C00E94250AF801738323
:102DD00062838FED93E0EDDC83EE93E0EADC60E06C
:102DE00070E0CB01EFDC89EE93E0E3DCC701B601D4
:102DF000E9DC8FEE93E0DDDCC501B401E3DC85EFB7
:102E000093E0D7DC4AE06D857E858F8598898EDCDE
:102E10008CEF93E0CEDC69817A818B819C81D2DC5E
:102E200082E094E0C6DC69857A858B859C85CADC66
:102E300088E094E0BEDC6D817E818F819885C2DC64
:102E40008EE094E0B6DC87EB93E0B3DC89899A8965
:102E5000E1DC8CE897E0ADDCF801E15AFF4F29890D
:102E60003A89C901B0E0A0E080839183A283B38353
:102E700060E0C8010E94190D882331F0F801FE9628
:102E8000108211821282138262960FB6F894DEBF0E
:102E90000FBECDBFDF91CF911F910F91FF90EF90AB
:102EA000DF90CF90BF90AF909F908F907F906F906A
:102EB0005F904F903F902F9008952D853E854F85D0
:102EC00058892C153D054E055F0508F453C08981CE
:102ED0009A81AB81BC818C159D05AE05BF055CF464
:102EE000AD81BE811196BA8BA98B81E0F3018083FD
:102EF000D1018C9350CFC701B6010E942E4F2B01F8
:102F00003C0169817A818B819C810E942E4F9B01BB
:102F1000AC01C301B2010E941C512B013C016D8127
:102F20007E818F81988529853A854B855C85621BDA
:102F3000730B840B950B0E942E4F9B01AC01C301B8
:102F4000B2010E948D4F2B013C0169857A858B85EA
:102F50009C850E942E4F9B01AC01C301B2010E94CF
:102F6000B8500E9484517A8B698B81E0F801E9594D
:102F7000FF4FBDCFD501C40129813A814B815C81CE
:102F8000821B930BA40BB50BC816D906EA06FB06E9
:102F90005CF44D815E814E5F5F4F5A8B498B81E0BF
:102FA000F801E759FF4FA3CFC501B4016C197D09A2
:102FB0008E099F090E942E4F2B013C0169817A8165
:102FC0008B819C810E942E4F9B01AC01C301B201F9
:102FD0000E941C512B013C016D817E818F8198855F
:102FE00029853A854B855C85621B730B840B950B99
:102FF0000E942E4F9B01AC01C301B2010E948D4F74
:103000002B013C0169857A858B859C850E942E4F1A
:103010009B01AC01C301B2010E94B8500E948451CF
:103020007A8B698B81E0F801E859FF4F60CF4F92AE
:103030005F926F927F928F929F92AF92BF92CF9248
:10304000DF92EF92FF920F931F93CF936B017C015E
:10305000742EAC019B010E94B951882391F084E148
:1030600094E0CF911F910F91FF90EF90DF90CF9060
:10307000BF90AF909F908F907F906F905F904F9098
:1030800048CB46015701E894B7F82FEF3FEF4FE7E1
:103090005FE7C501B4010E94B95181110DC02FEF46
:1030A0003FEF4FE75FE7C501B4010E94284F1816B4
:1030B0001CF488E194E0D5CF2FEF3FEF4FE75FE4BA
:1030C000C701B6010E94B55118161CF48CE194E0BA
:1030D000C8CF2FEF3FEF4FE75FECC701B6010E946B
:1030E000284F87FDF3CF20E030E0A901C701B601EA
:1030F0000E94284F10E000E087FF08C08DE20E9488
:1031000079088C01F7FAF094F7F8F094C0E060E0E9
:1031100070E080E09FE37C1641F020E030E040E288
:1031200051E40E941C51CF5FF6CFA70196010E9487
:10313000B8502B013C010E9489514B015C014AE0CF
:10314000F5DA7C01E00EF11ECC23A9F1C501B40132
:103150000E942C4F9B01AC01C301B2010E94B750E9
:103160004B015C018EE20E947908E80EF91EC15005
:1031700010F120E030E040E251E4C501B4010E94CA
:103180008D4F2B013C010E9489514B01B12CA12C88
:103190004AE0C501B401CADAE80EF91EC501B4015E
:1031A0000E942C4F9B01AC01C301B2010E94B75099
:1031B0004B015C01DCCFC701CF911F910F91FF90B4
:1031C000EF90DF90CF90BF90AF909F908F907F90C7
:1031D0006F905F904F900895CF92DF92EF92FF92A1
:1031E000CF93DF93EC0188819981AA81BB81181666
:1031F00019061A061B0644F081E090E0A0E0B0E05A
:1032000088839983AA83BB838C819D81AE81BF8192
:10321000181619061A061B0644F081E090E0A0E09B
:10322000B0E08C839D83AE83BF8388859985AA8512
:10323000BB85181619061A061B0644F081E090E0BB
:10324000A0E0B0E088879987AA87BB8780E294E0F6
:10325000B0DA85E394E0ADDA6091DC087091DD08C6
:103260008091DE089091DF080E942E4F6B017C0157
:10327000688179818A819B810E942E4F9B01AC01DC
:10328000C701B6010E941C5142E0D1DE85E494E002
:1032900090DA6091E0087091E1088091E2089091E5
:1032A000E3080E942E4F6B017C016C817D818E8131
:1032B0009F810E942E4F9B01AC01C701B6010E9465
:1032C0001C5142E0B4DE85E594E073DA6091E408D5
:1032D0007091E5088091E6089091E7080E942E4FD2
:1032E0006B017C01688579858A859B850E942E4FBC
:1032F0009B01AC01C701B6010E941C5142E097DE60
:10330000DF91CF91FF90EF90DF90CF9088CAA2D845
:1033100063DF90E080E008958F929F92AF92BF921A
:10332000CF92DF92EF92FF920F931F93CF93DF9391
:10333000EC0186E292E03DDA85E394E03ADA6E0150
:1033400086E7C81A8EEFD80AC6010E949B0F0E941A
:103350002E4F4B015C01FE01ED55FD4F60817181E7
:10336000828193810E942E4F9B01AC01C501B40163
:103370000E941C5142E05BDE85E494E01ADA7E0193
:10338000E6E4EE1AEEEFFE0AC7010E949B0F0E94D0
:103390002E4F4B015C01FE01E955FD4F60817181AB
:1033A000828193810E942E4F9B01AC01C501B40123
:1033B0000E941C5142E03BDE85E594E0FAD98E0183
:1033C00006511E4FC8010E949B0F0E942E4F4B01B9
:1033D0005C01C555DD4F688179818A819B810E949E
:1033E0002E4F9B01AC01C501B4010E941C5142E06B
:1033F0001EDE30D814DA82E292E0DBD985E394E075
:10340000D8D9F601A68DB78D208931894289538993
:103410000E948050D7D985E494E0CBD9F701A68DDE
:10342000B78D20893189428953890E948050CAD939
:1034300085E594E0BED9F801A68DB78D2089318944
:10344000428953890E948050BDD904D8DF91CF9121
:103450001F910F91FF90EF90DF90CF90BF90AF90B2
:103460009F908F90DCC9CF92DF92EF92FF920F93E3
:103470001F93CF93DF938C016A017B01EC01CC0F8A
:10348000DD1F642FCE010E944C509927F7FC9A95BE
:103490008F2D7E2D6D2DCE0101960E944C500D5822
:1034A00011090330110588F4B701992777FD90952C
:1034B000892FCE0144960E944C506F2D7727882784
:1034C0009927CE0145960E944C5090E080E0DF9114
:1034D000CF911F910F91FF90EF90DF90CF900895C3
:1034E0004F925F926F927F928F929F92AF92BF9214
:1034F000CF92DF92EF92FF920F931F93CF93DF93C0
:103500008C01EC01CC0FDD1FCE010E944450882EAF
:10351000912CB12CA12CCE0101960E944450C82EB2
:10352000D12CF12CE12C0D5811090330110508F0B4
:103530005AC0CE0144960E944450482E512C712C02
:10354000612CCE0145960E944450082F10E030E0D7
:1035500020E08FEF481651046104710429F50F3FF4
:1035600011052105310501F58FEF88169104A1049D
:10357000B104C9F58FEFC816D104E104F10499F53F
:103580006FEF7FEFCB01DF91CF911F910F91FF90F4
:10359000EF90DF90CF90BF90AF909F908F907F90F3
:1035A0006F905F904F900895003811052105310507
:1035B0003CF7FE2CED2CDC2CCC24C701B601680DA9
:1035C000791D8A1D9B1D320155244424640D751DEF
:1035D000861D971D302F222711270027600F711F8E
:1035E000821F931FD0CF00E010E09801412C512C96
:1035F000320180E8C816D104E104F104D4F2C0CF4E
:10360000EF92FF920F931F93CF93DF938091C207A6
:103610009091C307892B51F584E090E00E94AF4957
:103620007C0190E080E05CDF1616170654F1C701BC
:103630000E943411D0E0C0E0CE010E94D001882366
:1036400069F0FE01EE0FFF1FEE0FFF1FEA50F74F6C
:103650004081518162817381CE0105DF2196C63997
:10366000D10551F7F092C307E092C2078091C207DB
:103670009091C307DF91CF911F910F91FF90EF9031
:10368000089583E090E02CDF61307105810591059C
:1036900031F506EF18E0D0E0C0E0CE010E94D00185
:1036A0008823B1F0CE011CDFF8016083718382832F
:1036B00093836F3F7F4F8F4F9F4F51F4CE010E94F6
:1036C0006602F8014081518162817381CE01CBDEB7
:1036D00021960C5F1F4FC13ED105F9F6C3CFC7013C
:1036E0000E943411BFCF8CDF09DA84E294E061D804
:1036F0000E942A1294D890E080E00895CF92DF9241
:10370000EF92FF920F931F93CF93DF937C016B0196
:103710008A01E90175DFF601EE0FFF1FEE0FFF1FB3
:10372000EA50F74F80819181F7019183808368DFB0
:10373000000F111F000F111FF801EA50F74F81E031
:10374000408151816281738141305105610571056C
:1037500009F080E0F701828753DFCC0FDD1FCC0F2B
:10376000DD1FCA50D74F88819981AA81BB81F7019B
:1037700082839383A483B583168217821086118671
:10378000DF91CF911F910F91FF90EF90DF90CF903D
:103790000895CF93DF93EC012AEC30E04BEC50E03E
:1037A00069EC70E0ABDF2EEC30E04FEC50E06DECFC
:1037B00070E0CE010C96A2DF24ED30E045ED50E044
:1037C00063ED70E0CE01489699DF28ED30E049EDD9
:1037D00050E067ED70E0CE01849690DF2EED30E092
:1037E0004FED50E06DED70E0CE01C096DF91CF91CE
:1037F00085CFCF93DF938091C9079091CA07892B1A
:10380000A1F48CE390E00E94AF49EC011982188288
:103810001D861C86198E188E1DA21CA219AA18AA14
:10382000B8DFD093CA07C093C9078091C9079091A8
:10383000CA07DF91CF9108952F923F924F925F92E6
:103840006F927F928F929F92AF92BF92CF92DF92B0
:10385000EF92FF920F931F93CF93DF93EC01D0DE93
:10386000FE01E752FD4F8091B20A9091B30A918315
:103870008083C6DEFE01E552FD4F8091B60A90912D
:10388000B70A91838083BCDEFE01E352FD4F809135
:10389000BA0A9091BB0A91838083B2DE8E010152F5
:1038A0001D4F6091DA0A7091DB0A8091DC0A9091D9
:1038B000DD0A0E942E4FF801608371838283938317
:1038C0009FDE1E01FDE12F1AFDEF3F0A6091DE0A27
:1038D0007091DF0A8091E00A9091E10A0E942E4FD8
:1038E000F10160837183828393838ADE20E030E07C
:1038F00048EC52E4F80160817181828193810E94D9
:103900001C512B013C0120E030E048EC52E4F10175
:1039100060817181828193810E941C514B015C0105
:103920006091E20A7091E30A8091E40A9091E50ABD
:103930000E942E4F20E030E048EC52E40E941C51DF
:103940006B017C012AE037ED43E25CE3C301B20185
:103950000E94B55118160CF02AC120E030E046EC68
:1039600052E4C301B2010E94284F87FD06C0412CDA
:10397000512C56EC652E52E4752EF801408251828E
:10398000628273822AE037ED43E25CE3C501B40151
:103990000E94B55118160CF013C120E030E046EC3F
:1039A00052E4C501B4010E94284F87FD06C0812C56
:1039B000912C36ECA32E32E4B32EF1018082918259
:1039C000A282B3822AE037ED43E25CE3C701B6018D
:1039D0000E94B55118160CF0FCC020E030E046EC17
:1039E00052E4C701B6010E94284F87FD06C0C12CD2
:1039F000D12C96ECE92E92E4F92EFE01E951FD4F0F
:103A0000C082D182E282F382FBDD80919A0A90919A
:103A10009B0AFE01E251FD4F91838083F1DD80918D
:103A20009E0A90919F0AFE01E051FD4F9183808391
:103A3000E7DD8091A20A9091A30AFE01EE50FD4FAE
:103A400091838083DDDD8091C20A9091C30AA091A9
:103A5000C40AB091C50AFE01EC50FD4F80839183EA
:103A6000A283B383CDDD8091C60A9091C70AA0914D
:103A7000C80AB091C90AFE01E850FD4F80839183C6
:103A8000A283B383BDDD8091CA0A9091CB0AA09135
:103A9000CC0AB091CD0AFE01E450FD4F80839183A2
:103AA000A283B383ADDD8091EA0A9091EB0AFE0117
:103AB000FD5F91838083A4DD8091EE0A9091EF0AEF
:103AC000FE01EE5FFC4F918380839ADD8091F20AC4
:103AD0009091F30AFE01EC5FFC4F9183808390DDAF
:103AE0008091020B9091030BFE01EA5FFC4F9183E2
:103AF000808386DD8091060B9091070BFE01E85FC5
:103B0000FC4F918380837CDD80910A0B90910B0B9D
:103B1000FE01E65FFC4F9183808372DD80918A0A0B
:103B200090918B0AA0918C0AB0918D0AFE01E5510B
:103B3000FD4F0197A105B10509F054C081E08083D4
:103B40005FDD80918E0A90918F0AA091900AB091CA
:103B5000910AFE01E451FD4F0197A105B10509F05D
:103B600043C081E080834CDD8091920A9091930A5A
:103B7000A091940AB091950AC351DD4F0197A10518
:103B8000B105A1F581E08883DF91CF911F910F915D
:103B9000FF90EF90DF90CF90BF90AF909F908F906D
:103BA0007F906F905F904F903F902F9008954AE0E4
:103BB000442E47ED542E43E2642E4CE3742EDDCEAA
:103BC0002AE0822E27ED922E23E2A22E2CE3B22EA3
:103BD000F4CE8AE0C82E87EDD82E83E2E82E8CE35F
:103BE000F82E0BCF1082ACCF1082BDCF1882CCCF75
:103BF0002F923F924F925F926F927F928F929F92FD
:103C0000AF92BF92CF92DF92EF92FF920F931F93EA
:103C1000CF93DF93CDB7DEB765970FB6F894DEBFCD
:103C20000FBECDBF998B888BEBDCE889F989EF5CFF
:103C3000FD4F81E04091C2095091C3096091C409D0
:103C40007091C509452B462B472B09F480E08083F2
:103C5000D7DCE889F989EE5CFD4F81E04091C60927
:103C60005091C7096091C8097091C909452B462B2D
:103C7000472B09F480E08083C3DCE889F989ED5C97
:103C8000FD4F81E04091CA095091CB096091CC0968
:103C90007091CD09452B462B472B09F480E080839A
:103CA000AFDC8091120A9091130AA091140AB0918E
:103CB000150AE889F989EC5CFD4F80839183A28322
:103CC000B3839EDC8091160A9091170AA091180A7E
:103CD000B091190AE889F989E85CFD4F80839183E6
:103CE000A283B3838DDC80911A0A90911B0AA09164
:103CF0001C0AB0911D0AE889F989E45CFD4F8083B4
:103D00009183A283B3837CDC8091EA099091EB09D3
:103D1000A091EC09B091ED09E889F989E45BFD4FC8
:103D200080839183A283B3836BDC8091EE099091B1
:103D3000EF09A091F009B091F109E889F989E05BF8
:103D4000FD4F80839183A283B3835ADC8091F20973
:103D50009091F309A091F409B091F509E889F989E6
:103D6000EC5AFD4F80839183A283B38349DC809119
:103D7000FA099091FB09A091FC09B091FD09E8892D
:103D8000F989E85AFD4F80839183A283B38338DC9D
:103D90008091FE099091FF09A091000AB091010A5B
:103DA000E889F989E45AFD4F80839183A283B38324
:103DB00027DC8091020A9091030AA091040AB09135
:103DC000050AE889F989E05AFD4F80839183A2832F
:103DD000B38316DC80919A0990919B09A0919C096C
:103DE000B0919D09E889F989EC59FD4F8083918351
:103DF000A283B38305DC80919E0990919F09A091D5
:103E0000A009B091A109E889F989E859FD4F80839B
:103E10009183A283B383F4DB8091A2099091A309DB
:103E2000A091A409B091A509E889F989E459FD4F49
:103E300080839183A283B383E3DBE889F989E05926
:103E4000FD4F81E0209172093091730921303105D5
:103E500009F080E08083D4DBE889F989EF58FD4FD1
:103E600081E020917609309177092130310509F000
:103E700080E08083C5DBE889F989EE58FD4F81E059
:103E800020917A0930917B092130310509F080E0D9
:103E90008083B6DBE889F989E257FD4F81E04091E4
:103EA0004A0950914B0960914C0970914D09452B7D
:103EB000462B472B09F480E08083A2DBE889F9894F
:103EC000E157FD4F81E040914E0950914F096091BB
:103ED000500970915109452B462B472B09F480E07E
:103EE00080838EDBE889F989E057FD4F81E04091BE
:103EF0005209509153096091540970915509452B0D
:103F0000462B472B09F480E080837ADBE889F98926
:103F1000EF56FD4F81E04091220A5091230A6091B3
:103F2000240A7091250A452B462B472B09F480E083
:103F3000808366DBE889F989EE56FD4F81E0409188
:103F4000260A5091270A6091280A7091290A452B68
:103F5000462B472B09F480E0808352DBE889F989FE
:103F6000ED56FD4F81E040912A0A50912B0A609155
:103F70002C0A70912D0A452B462B472B09F480E023
:103F800080833EDBE889F989EC56FD4F81E0209182
:103F90005A0930915B092130310509F080E08083B6
:103FA0002FDBE889F989EB56FD4F81E020915E090E
:103FB00030915F092130310509F080E0808320DBFA
:103FC000E889F989EA56FD4F81E020916209309134
:103FD00063092130310509F080E0808311DB809195
:103FE000220990912309A0912409B0912509E8891B
:103FF000F989E956FD4F80839183A283B38300DB67
:104000008091260990912709A0912809B09129094A
:10401000E889F989E556FD4F80839183A283B383B4
:10402000EFDA80912A0990912B09A0912C09B09187
:104030002D09E889F989E156FD4F80839183A28398
:10404000B383DEDAE889F989EE57FD4F81E04091CC
:104050003209509133096091340970913509452B2B
:10406000462B472B09F480E08083CADAE889F98976
:10407000ED57FD4F81E0409136095091370960912D
:10408000380970913909452B462B472B09F480E0FC
:104090008083B6DAE889F989EC57FD4F81E04091D9
:1040A0003A0950913B0960913C0970913D09452BBB
:1040B000462B472B09F480E08083A2DA80912A0BFB
:1040C00090912B0BA0912C0BB0912D0BE889F989C5
:1040D000ED58FD4F80839183A283B38391DA809161
:1040E0002E0B90912F0BA091300BB091310BE889E2
:1040F000F989E958FD4F80839183A283B38380DAE5
:104100008091320B9091330BA091340BB091350B11
:10411000E889F989E558FD4F80839183A283B383B1
:104120006FDAE889F989EB57FD4F81E020918A0920
:1041300030918B092130310509F080E08083E889D6
:10414000F989EA57FD4F1082E889F989E957FD4F4F
:10415000108256DAE889F989E857FD4F81E020910D
:104160008609309187092130310509F080E080838C
:10417000E889F989E757FD4F1082E889F989E65700
:10418000FD4F10823DDAE889F989E557FD4F81E05E
:104190002091AA093091AB092130310509F080E066
:1041A00080832EDAE889F989E457FD4F81E0209178
:1041B000AE093091AF092130310509F080E08083EC
:1041C0001FDAE889F989E357FD4F81E02091B209B0
:1041D0003091B3092130310509F080E0808310DA95
:1041E000E889F989E158FD4F81E020913A0B30913F
:1041F0003B0B2130310509F080E0808301DAE8894A
:10420000F989E058FD4F81E020913E0B30913F0B42
:104210002130310509F080E08083F2D9E889F989FD
:10422000EF57FD4F81E02091420B3091430B21303D
:10423000310509F080E08083E3D9088919890D559B
:104240001D4F8091D2099091D309A091D409B091CA
:10425000D509F80180839183A283B383D1D9E888FB
:10426000F988F9E5EF1AFDEFFF0A8091D6099091E0
:10427000D709A091D809B091D909F701808391831A
:10428000A283B383BDD98091DA099091DB09A09113
:10429000DC09B091DD09C888D988F5E5CF1AFDEFB2
:1042A000DF0AF60180839183A283B383F801408102
:1042B000518162817381141615061606170644F0A3
:1042C00041E050E060E070E040835183628373839B
:1042D000F70140815181628173811416150616061B
:1042E000170644F041E050E060E070E04083518305
:1042F00062837383181619061A061B064CF081E0B8
:1043000090E0A0E0B0E0F60180839183A283B383C4
:104310000E942A12FC01D6018D909D90AD90BC9018
:10432000D7014D915D916D917C91D8010D911D91B9
:104330002D913C91008311832283338344835583E1
:104340006683778380869186A286B386E889F98919
:104350007096FB83EA83E889F989E158FD4F208153
:104360002983E889F989ED58FD4F80819181A281E7
:10437000B381E889F989E557FD4F20812D83E889CC
:10438000F989EC56FD4F20812C83E889F989EB5798
:10439000FD4F20812987E889F989E857FD4F208161
:1043A0002A87E889F989EF56FD4F20812E87E88911
:1043B000F989E257FD4F20812F87E889F989E05973
:1043C000FD4F2080E889F989EF5CFD4F3080E88956
:1043D000F989E956FD4F4081518162817381E889F5
:1043E000F989EC59FD4F0081118122813381E889DF
:1043F000F989E85AFD4FC080D180E280F380E889D6
:10440000F989E45BFD4F80809180A280B380E889C8
:10441000F989EC5CFD4F4080518062807380E889AF
:10442000F98940A651A662A673A684A695A6A6A65B
:10443000B7A6C0AAD1AAE2AAF3AA04AB15AB26ABD1
:1044400037AB40AF51AF62AF73AF34AE25AE2F85FF
:1044500025A32E8526A32C8127A340E450E060E00D
:1044600070E0E05CFF4F40835183628373832A8551
:10447000E889F98926AF298527AFEC5BFF4F2D81AD
:104480002083E889F989EB5BFF4F80839183A283C6
:10449000B383E889F989E75BFF4F89818083A88925
:1044A000B98955968D919C9156978633910509F05F
:1044B00033C287E09CE0FD01E258FF4F9183808387
:1044C00032961182108285E09CE03696918380833B
:1044D000329611821082E889F989838D948D4A97EA
:1044E000D1F483E09CE0EE57FF4F91838083E8890D
:1044F000F989EC57FF4F1182108281E09CE0E88936
:10450000F989E657FF4F91838083E889F989E45759
:10451000FF4F118210820889198902571F4FE889BD
:10452000F989E058FD4F20812983E889F989E95804
:10453000FD4F80819181A281B3818D839E83AF8362
:10454000B887E889F989E457FD4F90819C83E88911
:10455000F989EB56FD4FA081A987E889F989EA57C7
:10456000FD4FB081BA87E889F989E757FD4F20816F
:104570002E87E889F989EE56FD4F2080E889F98970
:10458000E157FD4F3080E889F989EF58FD4F3081C0
:10459000E889F989EE5CFD4F2081E889F989E556C3
:1045A000FD4F80819181A281B381E889F989E85921
:1045B000FD4F4081518162817381E889F989E45A14
:1045C000FD4FC080D180E280F380E889F989E05B0B
:1045D000FD4F80809180A280B380E889F989E85CF2
:1045E000FD4F4080518062807380F801408E518E73
:1045F000628E738E848E958EA68EB78EC0A2D1A247
:10460000E2A2F3A244A355A366A377A380A791A730
:10461000A2A7B3A724A735A7358A268A2985278B81
:1046200080E490E0A0E0B0E080AB91ABA2ABB3AB94
:104630002E8526A78A8587A79C8194AB8D819E8134
:10464000AF81B88585AB96ABA7ABB0AF298121AF61
:10465000858196818633910509F090C187E09CE0C1
:10466000E889F989E450FF4F91838083E889F989CB
:10467000E250FF4F1182108285E09CE0E889F989C1
:10468000EC5FFE4F91838083E889F989EA5FFE4FF2
:1046900011821082D8011B968D919C914A97D9F472
:1046A00083E09CE0E889F989F39591838083E88928
:1046B000F989EE5FFE4F1182108281E09CE0E8896B
:1046C000F989E85FFE4F91838083E889F989E65F85
:1046D000FE4F11821082E888F988B4EFEB1ABEEF22
:1046E000FB0AE889F989EF57FD4F20812983E88982
:1046F000F989E558FD4F80819181A281B3818D8335
:104700009E83AF83B887E889F989E357FD4F90818D
:104710009C83E889F989EA56FD4F3080E889F98958
:10472000E957FD4FA081A987E889F989E657FD4F30
:104730002080E889F989ED56FD4FC080E889F98924
:10474000E057FD4FD080E889F989EE58FD4F308160
:10475000E889F989ED5CFD4F2081E889F989E15606
:10476000FD4F80819181A281B3818A8B9B8BAC8B21
:10477000BD8BE889F989E459FD4F408151816281FF
:104780007381E889F989E05AFD4F80809180A28089
:10479000B380E889F989EC5AFD4F408051806280EE
:1047A0007380E889F989E45CFD4F80819181A28161
:1047B000B381F701808F918FA28FB38F448E558E76
:1047C000668E778E80A291A2A2A2B3A244A355A323
:1047D00066A377A38A899B89AC89BD8980A791A7A5
:1047E000A2A7B3A724A735A7D58AC68A378A80E4AB
:1047F00090E0A0E0B0E080AB91ABA2ABB3AB26A65B
:10480000298527A78C8184AB8D819E81AF81B88556
:1048100085AB96ABA7ABB0AF298121AF85819681DF
:104820008633910509F0D2C087E09CE0E889F989D8
:10483000E658FE4F91838083E889F989E458FE4F5A
:104840001182108285E09CE0E889F989EE57FE4FDD
:1048500091838083E889F989EC57FE4F1182108299
:10486000D7011B968D919C914A97E1F483E09CE0DF
:10487000E889F989E258FE4F91838083E889F989B4
:10488000E058FE4F1182108281E09CE0E889F989AE
:10489000EA57FE4F91838083E889F989E857FE4FF4
:1048A00011821082E889F989EE57FD4F80818823B3
:1048B00009F4B4C08A819B810E948E0CE889F98931
:1048C000ED57FD4F8081882309F4ADC0C8010E94D7
:1048D0008E0CE889F989EC57FD4F8081882309F413
:1048E000A6C0C70165960FB6F894DEBF0FBECDBF58
:1048F000DF91CF911F910F91FF90EF90DF90CF90BC
:10490000BF90AF909F908F907F906F905F904F90EF
:104910003F902F900C948E0C8C339105D9F48FEF2F
:104920009BE0E889F989E258FF4F91838083E88909
:10493000F989E058FF4F118210828DEF9BE0E889E2
:10494000F989EA57FF4F91838083E889F989E8570D
:10495000FF4FBFCD8E9709F0BECD87EF9BE0E88972
:10496000F989E258FF4F91838083E889F989E058FB
:10497000FF4F1182108281EF9BE0E1CF8C339105D4
:1049800089F48FEF9BE0E889F989E450FF4F918328
:104990008083E889F989E250FF4F118210828DEF00
:1049A0009BE06CCE8E9709F075CE87EF9BE0E8898F
:1049B000F989E450FF4F91838083E889F989E250B7
:1049C000FF4F1182108281EF9BE058CE8C3391050E
:1049D00089F48FEF9BE0E889F989E658FE4F9183CF
:1049E0008083E889F989E458FE4F118210828DEFA7
:1049F0009BE02ACF8E9709F033CF87EF9BE0E889C1
:104A0000F989E658FE4F91838083E889F989E45853
:104A1000FE4F1182108281EF9BE016CF8A819B812D
:104A20000E947C0C4BCFC8010E947C0C52CFC70166
:104A300065960FB6F894DEBF0FBECDBFDF91CF9164
:104A40001F910F91FF90EF90DF90CF90BF90AF90AC
:104A50009F908F907F906F905F904F903F902F909E
:104A60000C947C0CAF92BF92CF92DF92EF92FF92A8
:104A70000F931F93CF93DF93EC0186E390E09E8B1F
:104A80008D8B87E390E0988F8F8B86E290E09A8FF2
:104A9000898F8AE190E09C8F8B8F8CE190E09E8FD4
:104AA0008D8F88E190E098A38F8F83E090E09AA3A8
:104AB00089A382E090E09CA38BA3FE01E257FF4F05
:104AC0008CE390E0968385838DE390E090878783E5
:104AD00088E390E092878187148613861686158670
:104AE000108A17868EE090E0928B818B8FE090E0A9
:104AF000948B838BE258FF4F8EE290E09683858300
:104B000080E390E0908787838EE390E092878187AF
:104B10001486138616861586108A178682E190E021
:104B2000928B818B83E190E0948B838BE15EFE4FCF
:104B30001182108232961182108232961182108276
:104B4000CE0156D8CE010E941C1C6E0186E7C81A01
:104B50008EEFD80AAA24A394B12CF601B7A6A6A674
:104B60007E01F6E4EF1AFEEFFF0A84E090E0F70121
:104B700097A786A78E0106511E4F88E090E0F801A6
:104B800097A786A780E190E0F6019183808381E179
:104B900090E0958384838FE190E09383828381E228
:104BA00090E097838683C6010E94390FF6018285C3
:104BB00080878385818787E190E0F70191838083F7
:104BC00089E190E09583848383E290E093838283FC
:104BD00085E290E097838683C7010E94390FF70131
:104BE00082858087838581878BE190E0F8019183BE
:104BF00080838DE190E09583848387E290E09383C6
:104C0000828389E290E097838683C8010E94390FEE
:104C1000F8018285808783858187E45EFE4F8081ED
:104C20009181729740815181628173813697208191
:104C30003181F601358F248F448B558B668B778BB2
:104C4000019709F044C08FEF9FEF978F868FFE0189
:104C5000E85FFC4F80819181709740815181628132
:104C60007381389720813181F701358F248F448BF0
:104C7000558B668B778B019769F58FEF9FEF978F39
:104C8000868FFE01E65FFC4F808191813E974081D7
:104C9000518162817381CE50DD4F28813981F801C5
:104CA000358F248F448B558B668B778B0197A9F4B6
:104CB0008FEF9FEF978F868FDF91CF911F910F918D
:104CC000FF90EF90DF90CF90BF90AF900895B78E98
:104CD000A68EBDCF81E090E0D2CF81E090E0EACF18
:104CE000CF92DF92EF92FF920F931F93CF93DF93B8
:104CF0008B010E94001BEC01F801C2A0D3A0E4A02C
:104D0000F5A0068D178D8A819B818F30F7E29F0772
:104D10005CF501969B838A83C8010E94D001882399
:104D200031F1F801EE0FFF1FEE0FFF1FEA50F74FB2
:104D3000C082D182E282F382B701A601C8010E943B
:104D4000331AB801CE010E9444150E94F91B0E943B
:104D5000C91B90E080E0DF91CF911F910F91FF90F0
:104D6000EF90DF90CF9008951B821A82D5CF8DEB04
:104D700093E00E94D913E9CFCF93DF93EB010E9418
:104D8000001B6E8D7F8D0E94441590E080E0DF91C6
:104D9000CF910895FC0180819181009711F00C94CE
:104DA0004B4A08950C944B4A0C944B4A0C944B4A32
:104DB0000C944B4A0C944B4A0C944B4A0C944B4A1F
:104DC0000C944B4A0C944B4A0C944B4A0C944B4A0F
:104DD0000C944B4A0C944B4A0C944B4A0C944B4AFF
:104DE0000C944B4A0C944B4A0C944B4A0C944B4AEF
:104DF0000C944B4A0C944B4A0C944B4A0C944B4ADF
:104E00000F931F93CF93DF93EC01888199810097D3
:104E100059F02A813B812617370730F081E0DF9176
:104E2000CF911F910F9108958B016F5F7F4F0E946B
:104E3000E051009759F0998388831B830A832C8162
:104E40003D81232B59F7FC011082E8CF80E0E7CFAA
:104E50000F931F93CF93DF93EC018B01D1DF288158
:104E60003981811112C02115310519F0C9010E9443
:104E70004B4A198218821D821C821B821A82CE0123
:104E8000DF91CF911F910F9108951D830C836EE8E0
:104E900077E0C9010E94D152F2CFCF93DF93FC019A
:104EA000E25EFD4F408151814115510501F1EC0158
:104EB000CE5DDD4F28813981865E9D4F24173507F1
:104EC000E8F4FC01808191810097A1F0820F931F8B
:104ED000FC0180818A3031F08D3069F48CE897E0F4
:104EE0000E94D91388819981019699838883DF91E3
:104EF000CF91089580E00E947908F4CF70E060E0DF
:104F0000A7DF19821882F3CF2F923F924F925F92C0
:104F10006F927F928F929F92AF92BF92CF92DF92C9
:104F2000EF92FF920F931F93CF93DF93CDB7DEB72E
:104F3000CE57D1090FB6F894DEBF0FBECDBF8C019E
:104F4000FC01108211821282138214821582168251
:104F50001782108611861286138614861586168689
:104F600017864C01F0E18F0E911CC4010E94700E57
:104F700068018EE8C80ED11CC6010E94700E78012F
:104F8000E4EFEE1AEEEFFE0AC7010E94700E580120
:104F9000F6E7AF1AFEEFBF0AC5010E94FD0F380108
:104FA00086E4681A8EEF780AC3010E94FD0F28017B
:104FB000E6E14E1AEEEF5E0AC2010E94FD0FF80113
:104FC000E65EFD4F118210821382128215821482D6
:104FD00070E060E0CF013CDFF801E05EFD4F118240
:104FE000108232961182108232961182108232968D
:104FF0001182108232961082319610823196108280
:10500000319611821082329611821082329611826C
:10501000108232961082319610823196108231962B
:1050200010821182128213823496108211821282AF
:105030001382349610821182128213823496108267
:10504000118212821382349610821182128213828C
:105050003496108211821282138234961082118249
:105060001282138234961082118212821382349635
:10507000108211821282138234961082118212825F
:105080001382349610821182128213823496108217
:10509000118212821382349610821182128213823C
:1050A00034961082118212821382349610821182F9
:1050B00012821382349610823196108231961082B9
:1050C00031961082118212821382349610821182DC
:1050D00012821382349610821182128213823496C5
:1050E000108231961082319610823196108231965C
:1050F000108231961082319610823196108231964C
:10510000108231961082319610823196108231963B
:10511000108231961082319610823196108231962B
:10512000108231961082319610823196108231961B
:10513000108231961082319610823196108231960B
:10514000108211821282138234961082118212828E
:10515000138234961082118212821382D801AD55C7
:10516000BD4F8CE0E1E1F2E001900D928A95E1F70C
:10517000F801E155FD4F108211821282138234969C
:10518000108211821282138234961082118212824E
:1051900013823496118210823296118210823296D6
:1051A00011821082329610821182128213823496FA
:1051B000108211821282138234961082118212821E
:1051C00013823496108211821282138234961082D6
:1051D00011821282138234961082118212821382FB
:1051E0003496118210823296118210823296118288
:1051F00010823296108211821282138234961082AB
:1052000011821282138234961082118212821382CA
:105210003496108231961082319610823196118226
:10522000108232961182108232961182108232964A
:10523000108211821282138234961082118212829D
:105240001382349610821182128213823496118254
:10525000108232961182108232961182108232961A
:10526000118210823296118210823296118210823F
:105270003296118210823296118210821801F0EF5C
:105280002F1AFCEF3F0AF101108231961182108231
:10529000329611821082CE0101960E94700E8EE726
:1052A000FE013196D40101900D928A95E1F7CE016D
:1052B00001960E94700E8EE7FE013196D601019094
:1052C0000D928A95E1F7CE0101960E94700E8EE74D
:1052D000FE013196D70101900D928A95E1F788E59C
:1052E000F801808B89E5F60180838AE5F7018083E8
:1052F000CE0101960E94FD0F80E3FE013196D5019B
:1053000001900D928A95E1F7CE0101960E94FD0F62
:1053100080E3FE013196D30101900D928A95E1F769
:10532000CE0101960E94FD0F80E3FE013196D2016D
:1053300001900D928A95E1F7C80194DBF10110828A
:10534000C258DF4F0FB6F894DEBF0FBECDBFDF915E
:10535000CF911F910F91FF90EF90DF90CF90BF9072
:10536000AF909F908F907F906F905F904F903F9005
:105370002F900895CF93DF938091C0079091C1073C
:10538000892B51F485E193E00E94AF49EC01BCDD2B
:10539000D093C107C093C0078091C0079091C10707
:1053A000DF91CF9108950F93CF93DF938091C6073C
:1053B00081114CC081E08093C607DCDFEC0106B1AF
:1053C00026B140910001609100010295017026FB19
:1053D000222720F941706695617086579E4F0E9482
:1053E0006C0F06B126B140B160B1017022FB2227DB
:1053F00020F943FB442740F966956170CE0186543D
:105400009E4F0E946C0F02B322B340B160B1017095
:1054100022FB222720F9441F4427441F65FB6627EF
:1054200060F9CE0186519E4F0E946C0FCE014096CE
:105430000E943C0ECE0182579F4F0E943C0ECE012F
:10544000845F9E4F0E943C0E1092C607DF91CF9161
:105450000F910895CF93DF93EB0120E030E040E817
:105460005FE36A817B818C819D810E94284F81113D
:1054700013C088E294E00E94D9137CDFFC01E25B58
:10548000FF4F108211821282138286579E4FFC01B9
:10549000108A118A128A138A20E030E040E85FE324
:1054A0006E817F81888599850E94284F811113C064
:1054B00088E394E00E94D9135DDFFC01E453FF4FC1
:1054C000108211821282138286549E4FFC01108A30
:1054D000118A128A138A20E030E040E85FE36A858F
:1054E0007B858C859D850E94284F811113C088E49F
:1054F00094E00E94D9133EDFFC01E65BFE4F108270
:1055000011821282138286519E4FFC01108A118AE9
:10551000128A138A0E942A120E940F1490E080E0DF
:10552000DF91CF910895EF92FF920F931F93CF9346
:10553000DF936115710541F480E0DF91CF911F91F8
:105540000F91FF90EF90089541155105A9F07B014F
:10555000EC010C811D81040F151FB80151DC88235B
:1055600059F3288139818C819D81B701820F931F66
:105570000E94D1521D830C8381E0DFCFEF92FF9216
:105580000F931F93CF93DF93CDB7DEB764970FB61A
:10559000F894DEBF0FBECDBF7C01CB01BA018E01F6
:1055A0000F5F1F4F22E044E00E949249FC010190EE
:1055B0000020E9F73197AF01481B590BBC01C70127
:1055C000B2DF64960FB6F894DEBF0FBECDBFDF9199
:1055D000CF911F910F91FF90EF900895FB010190E3
:1055E0000020E9F73197AF01461B570B9CCFEF9294
:1055F000FF920F931F93CF93DF93CDB7DEB72E9714
:105600000FB6F894DEBF0FBECDBF8C01FC01118236
:105610001082138212821582148270E060E018DC1E
:1056200068E873E0C801DADF60917A0C70917B0C56
:1056300080917C0C90917D0C2AE0AE014F5F5F4F12
:105640007A010E940B4BF70101900020E9F7319796
:10565000AF014E195F09B701C80165DF6CE877E05B
:10566000C801BCDFC8012E960FB6F894DEBF0FBE8E
:10567000CDBFDF91CF911F910F91FF90EF900895D3
:10568000FB0144815581608171814DCFCF92DF92C2
:10569000EF92FF920F931F93CF93DF9300D000D030
:1056A0001F921F92CDB7DEB78B016A01865E9D4FB8
:1056B0007C016AE272E092DF67EB73E0C7018EDF84
:1056C000F801808189831A8241E050E08E010F5FEA
:1056D0001F4FB801C70127DF4AE0B801C6010E9489
:1056E000014BF80101900020E9F73197AF01401B11
:1056F000510BB801C70117DF0E942A12C80177DFDA
:10570000B801C701BDDFC80145DB28960FB6F89484
:10571000DEBF0FBECDBFDF91CF911F910F91FF90E4
:10572000EF90DF90CF9008952F923F924F925F922B
:105730006F927F928F929F92AF92BF92CF92DF92A1
:10574000EF92FF920F931F93CF93DF93CDB7DEB706
:10575000A3970FB6F894DEBF0FBECDBF9BA38AA35D
:105760007C836B830E94F81D8AA19BA10E941C1C54
:105770000E94B3120E9415152B813C81AAA0BBA0E8
:105780002130310509F464C02230310509F490C09C
:1057900030E1A30EB11C2AA03BA046E7241A4EEF2D
:1057A000340AEAA1FBA1E257FD4F508159878AA133
:1057B0009BA181559D4F9E838D83EAA1FBA1E7525A
:1057C000FD4FF98BE88B2AA13BA125513D4F3D8B25
:1057D0002C8B4AA15BA1455D5D4F5B874A878DE8B5
:1057E00090E09B8B8A8BE5E1F0E0F887EF83C501C1
:1057F0000E94410C882309F48AC088E594E00E9445
:10580000D9130E942A1281E090E090930C088093B3
:105810000B08E1E0F0E0FA83E98389819A81A3969D
:105820000FB6F894DEBF0FBECDBFDF91CF911F91B1
:105830000F91FF90EF90DF90CF90BF90AF909F902F
:105840008F907F906F905F904F903F902F90089532
:10585000FEE8AF0EB11C2AA03BA026E4221A2EEFD0
:10586000320AEAA1FBA1E157FD4F308139874AA1F5
:105870005BA14D545D4F5E834D838AA19BA18552F0
:105880009D4F998B888BEAA1FBA1E451FD4FFD8BC5
:10589000EC8B2AA13BA1235D3D4F3B872A874EE835
:1058A00050E05B8B4A8B86E190E098878F839FCF97
:1058B00094EFA91A9EEFB90A2AA03BA0E6E12E1A9E
:1058C000EEEF3E0AEAA1FBA1E057FD4F20812987B8
:1058D0004AA15BA149545D4F5E834D838AA19BA180
:1058E00083529D4F998B888BEAA1FBA1E351FD4F19
:1058F000FD8BEC8B2AA13BA1215D3D4F3B872A8785
:105900004FE850E05B8B4A8B87E190E0CECFC5013A
:105910000E94320C811171CF8FED93E00E94D91358
:105920008EE894E00E94D913F50180810E947908E5
:1059300085E994E00E94D9138CE897E00E94D9137E
:1059400081E090E0EA85FB859183808341E050E02F
:10595000B5018AA19BA19ADEC5010E948E0CF501BA
:1059600084A585010C591F4F882309F4B4C0C501D3
:105970000E94500CF8011082C1010E949B0FF5019A
:10598000FE966083718382839383ED81FE81108212
:10599000118212821382EAA1FBA1E155FD4F108210
:1059A000118212821382EAA1FBA1ED54FD4F1082F5
:1059B000118212821382EAA1FBA1E954FD4F1082E9
:1059C00011821282138286E090E0EA85FB85918342
:1059D000808346E050E0B5018AA19BA157DE61E0DB
:1059E00070E0C5010E941E148B809C80880C991C5D
:1059F000880C991CC40181529D4F2AA13BA1280FFC
:105A0000391F398F288F8B819C8180589E4F880F3A
:105A1000991F4AA15BA1480F591F5B8F4A8FC40190
:105A200083539D4FEAA1FBA1E80FF91FFD8FEC8F77
:105A30000C972AA13BA1280F391F3F8F2E8F429729
:105A40004AA15BA1480F591F59A348A3412C512CCF
:105A5000320143948B819C81EAA1FBA18E0F9F1F91
:105A60009C0125513D4F3F8B2E8BCF01880D991DF9
:105A7000AC01485A5D4F5D874C87EE89FF89808174
:105A8000882371F0C88CD98CEA8CFB8C0C8D1D8D11
:105A90002E8D3F8D48A159A1B101C5010E94481129
:105AA0008EE79CE00E94F60718161906DCF010E05D
:105AB0001A821982C5010E94410C882391F189EC58
:105AC00094E00E94D913C5010E94410C811101C0CC
:105AD000898589878DC0C5010E94660C81E0F80127
:105AE00080834ACF8EE79CE00E94D4078F7D853467
:105AF0009105E9F684EB94E00E94D9130E942A12E2
:105B000021E0FC01268786E592E00E94D9130E94DD
:105B10002A120E940F1441E050E05A83498311E099
:105B2000C9CFC5010E94320C8111C9CF1111C7CF55
:105B3000E889F98960817181072E000C880B990B27
:105B40000E942E4F9B01AC01ED81FE81608171812D
:105B5000828193810E94284F87FFB1CFC5010E94A7
:105B6000350DEC85FD85208131814281538160E5D1
:105B700073EC80E090E00E945A50C9010E94C40971
:105B8000EC85FD852081318142815381A3E0B0E025
:105B90000E9476509B01AC01C301B2010E945A5091
:105BA000672B682B692B41F482E592E00E94D913A0
:105BB0000E942A120E940F14C5010E94190CEC8544
:105BC000FD85208131814281538160E573EC80E065
:105BD00090E00E945A50C9010E94C409FFEF4F1A79
:105BE0005F0A6F0A7F0A29813A81232B09F445CF86
:105BF00062E070E0C5010E941E148FED93E00E94E8
:105C0000D9138EE894E00E94D913F50180810E9497
:105C100079088DED94E00E94D9138CE897E00E94FA
:105C2000D91329813A81232B09F580EF94E00E9452
:105C3000D91387EB93E00E94D9138FE893E00E9479
:105C4000D9138F8198850E940A1487EB93E00E94F4
:105C5000D9138DEB97E00E94D9133985832F90E0FB
:105C60000E940A140E942A120E940F140E94B3126A
:105C70000E9415158FED93E00E94D9138EE894E0F1
:105C80000E94D913F50180810E94790884EF94E085
:105C90000E94D9138CE897E00E94D913ED81FE8110
:105CA0001082118212821382F50184A585010C599C
:105CB0001F4F882309F41BC1C5010E94660C81E0B7
:105CC000F8018083C1010E949B0FF501FE9660835D
:105CD000718382839383EAA1FBA1E155FD4F10827A
:105CE000118212821382EAA1FBA1ED54FD4F1082B2
:105CF000118212821382EAA1FBA1E954FD4F1082A6
:105D0000118212821382C1010E949B0F6C877D87D2
:105D10008E879F87C1010E949B0F412C512C32011D
:105D20008B819C812AA13BA1820F931FAC0145511D
:105D30005D4F5F8B4E8B820E931EC401885A9D4F20
:105D400098878F834201E981FA81EF2B99F5EE89DB
:105D5000FF898081882371F0C88CD98CEA8CFB8CF8
:105D60000C8D1D8D2E8D3F8D48A159A1B101C5010E
:105D70000E9448118EE79CE00E94F607181619064B
:105D80000CF4BBC010E05AE08516910434F4ED81A8
:105D9000FE811082118212821382F985C501F111F0
:105DA00053C10E94410C882309F4C7C089EC94E0D8
:105DB0000E94D9138FED93E00E94D9138EE894E0EE
:105DC0000E94D913F50180810E94790886E195E04F
:105DD0000E94D9138CE897E00E94D913C1010E9458
:105DE0009B0F2C893D89232BA1F0DC01CB012C8555
:105DF0003D854E855F85821B930BA40BB50BB7FFCA
:105E000007C0B095A095909581959F4FAF4FBF4F1C
:105E10004C012401990C6608770849815A81452B69
:105E200019F580EF94E00E94D91387EB93E00E946C
:105E3000D9138FE893E00E94D9138A899B890E9425
:105E40000A1487EB93E00E94D9138DEB97E00E9430
:105E5000D913C301B2010E942E4F42E00E941718CD
:105E60000E942A120E940F1485E090E0EA85FB85CB
:105E70009183808345E050E0B5018AA19BA106DCB7
:105E8000C5010E947C0C0E94B3120E9415152B8143
:105E90003C812130310509F4C1C02230310509F4BB
:105EA000C8C00E942A124092DC085092DD0860921D
:105EB000DE087092DF080E942A120E94EC18EA8520
:105EC000FB851182108250E040E0B5018AA19BA1C0
:105ED000DDDB70E060E0C5010E941E140E942A1202
:105EE00029813A8130930C0820930B0896CCC50188
:105EF0000E94500CF8011082E5CE8EE79CE00E94D3
:105F0000D4078F7D8534910509F03CCF84EB94E074
:105F10000E94D9130E942A1221E0FC01268786E5FF
:105F200092E00E94D9130E942A120E940F1441E0AD
:105F300050E05A83498311E026CF111137CFE88909
:105F4000F98960817181072E000C880B990B0E94E2
:105F50002E4F9B01AC01ED81FE81608171818281B8
:105F600093810E94284F87FF21CFC5010E94350DE4
:105F70004201FFEF8F1A9F0AEF81F885208131815E
:105F80004281538160E573EC80E090E00E945A50BA
:105F9000C9010E94C409FFEF4F1A5F0A6F0A7F0A06
:105FA000EF81F8852081318142815381A3E0B0E007
:105FB0000E9476509B01AC01C301B2010E945A506D
:105FC000672B682B692BB9F482E592E00E94D91304
:105FD0000E942A120E940F148FED93E00E94D913A1
:105FE00088E095E00E94D913C4010E940A148CE84D
:105FF00097E00E94D913C5010E94190CEF81F88522
:10600000208131814281538160E573EC80E090E032
:106010000E945A50C9010E94C40994CE0E942A12BB
:106020004092E0085092E1086092E2087092E30822
:1060300042CF0E942A124092E4085092E5086092F2
:10604000E6087092E70837CF0E94320CACCEFA0116
:10605000DB01A959BF4F2C91222331F122E030E01E
:10606000DB01A759BF4F4C91442311F023E030E0EE
:10607000DB01A859BF4F4C91442311F024E030E0DC
:10608000DB01A659BF4F4C91442311F026E030E0CC
:10609000408151814217530761F0121613063CF4F8
:1060A00031832083A901F2CA30E020E0D9CF1182E8
:1060B000108208952F923F924F925F926F927F923B
:1060C0008F929F92AF92BF92CF92DF92EF92FF9208
:1060D0000F931F93CF93DF93CDB7DEB7E8970FB63B
:1060E000F894DEBF0FBECDBF1C012A013B010B8718
:1060F0001C872D873E8760960EAD1FAD6097FC0113
:10610000ED55FD4F60817181828193810E942E4FF8
:10611000A30192010E948D4F0E9484516B8F7C8F4E
:106120008D8F9E8FF101E955FD4F608171818281D4
:1061300093810E942E4F2B853C854D855E850E9464
:106140008D4F0E9484516BA37CA38DA39EA3F1016C
:10615000E555FD4F60817181828193810E942E4FB0
:10616000A70196010E948D4F0E9484516BA77CA7C6
:106170008DA79EA70E94250A6B877C878D879E87A7
:10618000F101EC5DFD4F1182108232961182108276
:106190003E96A114B10461F0C501B0E0A0E04081D9
:1061A00051816281738184179507A607B70714F0A0
:1061B000A080B180F101E85CFD4F80819181A281D6
:1061C000B3818114910441F0A40170E060E04817AC
:1061D00059076A077B070CF04C01F101E45CFD4FA5
:1061E00080819181A281B3810115110541F0A8013F
:1061F00070E060E0481759076A077B070CF08C01D4
:10620000210120E1420E511CC501B0E0A0E0F101E6
:1062100080A791A7A2A7B3A73101FEE86F0E711C5A
:10622000B12CA12CD30158968D929D92AD92BC9227
:106230005B974101B4EF8B1ABEEF9B0A30E020E080
:10624000F401008F118F228F338F0E942A120E9437
:106250002A120E942A120E942A122091DC083091F0
:10626000DD084091DE085091DF082B8B3C8B4D8B75
:106270005E8B0E942A128091E0089091E108A09123
:10628000E208B091E3088F87988BA98BBA8B0E94A4
:106290002A12A090E408B090E508C090E608D090DB
:1062A000E708F101E155FD4F10821182128213823D
:1062B00034961082118212821382349610821182D7
:1062C00012821382349611821082329611821082C9
:1062D00032961182108232962B893C894D895E89D3
:1062E000208331834283538334968F859889A9898B
:1062F000BA8980839183A283B3833496A082B182CA
:10630000C282D3826196EFAC61970B8D1C8D2D8D6F
:106310003E8D4B895C896D897E89C2010E94A10CEA
:106320008823F9F08EE492E00E94D91385E394E08B
:106330000E94D913F101EE5AFF4F60817181828171
:106340009381EF5AFD4F20813181428153810E9418
:106350005A50CA01B9010E94E2130E942A120E94F7
:106360000F146296EFAC62970BA11CA12DA13EA168
:106370004F85588969897A89C3010E94A10C8823B5
:10638000F9F08AE492E00E94D91385E494E00E9437
:10639000D913F101E053FF4F6081718182819381B4
:1063A000E952FE4F20813181428153810E945A502F
:1063B000CA01B9010E94E2130E942A120E940F141E
:1063C0006396EFAC63970BA51CA52DA53EA5B60162
:1063D000A501C4010E94A10C8823F9F086E492E093
:1063E0000E94D91385E594E00E94D913F101E25B84
:1063F000FE4F6081718182819381E35AFE4F20813B
:106400003181428153810E945A50CA01B9010E94D0
:10641000E2130E942A120E940F14D10151961C927D
:10642000F101E157FF4F1082E258FF4F10820E94A6
:10643000B3120E941515C2010E944F0EC3010E94A3
:106440004F0EC4010E944F0EF101E55DFD4FFCA708
:10645000EBA781E090E0918380837101F3EDEF1A67
:10646000FDEFFF0AD7018D939C938101015D1D4FC4
:10647000F8019183808341E050E0B201C10106D967
:10648000D7014D915C91B301C10100D9F801408160
:106490005181B401C101FAD811E0F101E05FFC4F74
:1064A0001083C2010E948E0CC3010E948E0CC40195
:1064B0000E948E0C64E670E080E090E00E94F40997
:1064C000C101885D9D4FDC011C9311961C93A101B5
:1064D000465D5D4FFA0110836196FFAD6197F11142
:1064E0000FC062962FAD6297211105C063963FAD34
:1064F0006397332339F191012D583F4FF9011082F1
:106500006296FFAD6297F11105C091012F503F4F88
:10651000F90110826396FFAD6397F11105C09101F7
:1065200021593E4FF901108261962FAD6197FC0110
:10653000208362963FAD62973C936396EFAD63977D
:10654000DA01EC93C2010E949615C3010E949615D0
:10655000C4010E949615C2010E94940DC3010E94BD
:10656000940DC4010E94940D0E942A12DC011E9613
:106570008C918F87B12CA12CF101E85DFD4FFC8B34
:10658000EB8B9101275D3D4F3C8F2B8FA101465D29
:106590005D4F5CA34BA3C101855D9D4F9CAB8BAB55
:1065A000D101A35DBD4FBEABADAB3796F8AFEFAB3E
:1065B0002D55314038AB2FA7405E51095AAB49AB3E
:1065C000AB89BC898C9181110AC0EB8DFC8D8081D7
:1065D000811105C0ABA1BCA18C91882319F0BF85A6
:1065E000BB2369F08101025E1D4FF801808191811A
:1065F000892B09F49FC4C1010E944D27F6CF4BA9F6
:106600005CA9B201C10123DD4DA95EA9B301C1019D
:106610001EDD4FA958ADB401C10119DDC2010E94B0
:10662000FC0DC3010E94FC0DC4010E94FC0DF10190
:10663000EA58FF4F8081882321F1C2010E949615FC
:10664000F101E551FD4F80818823B9F06101E1E25C
:10665000CE1AEDEFDE0A7101FDEFFF1A810103533F
:106660001D4F91012F533D4FA10141555D4FB10188
:1066700066577E4FC2010E944811F101EA58FF4F50
:106680001082F101EC50FF4F8081882331F1C3016A
:106690000E949615F101E451FD4F80818823C9F0D5
:1066A00061012DE1C21A2DEFD20A71013EEFE31A0A
:1066B0003CEFF30A81010F521D4F91012B533D4FC7
:1066C000A1014D545D4FB10166547E4FC3010E943C
:1066D0004811F101EC50FF4F1082F101EE58FE4FCE
:1066E0008081882329F1C4010E949615F101E351AC
:1066F000FD4F80818823C1F0610149E1C41A4DEF4B
:10670000D40A71015CEFE51AF50A81010B521D4FA5
:10671000910127533D4FA10149545D4FB10166518D
:106720007E4FC4010E944811F101EE58FE4F1082C5
:1067300081010D581F4FD8018C91882309F43EC068
:10674000F101E752FD4F60817181072E000C880B2B
:10675000990B0E942E4F9B01AC01F101E155FD4FB9
:1067600060817181828193810E94B551181634F540
:10677000F80110826FED73E009551E4FC8010E94A9
:10678000EE2A64E275E0C8010E94EE2A6CE877E028
:10679000C8010E94EE2A6196FFAD6197FF2309F4BC
:1067A0005BC1F101E657FE4F108A118A128A138AE3
:1067B000EC53F140108211821282138281010F503A
:1067C0001F4FD8018C91882309F43FC0F101E55295
:1067D000FD4F60817181072E000C880B990B0E9480
:1067E0002E4F9B01AC01F101ED54FD4F6081718191
:1067F000828193810E94B55118163CF5F8011082F0
:106800006FED73E0075D1E4FC8010E94EE2A6CE435
:1068100075E0C8010E94EE2A6CE877E0C8010E948A
:10682000EE2A6296FFAD6297FF2309F419C1F101C8
:10683000E654FE4F108A118A128A138AAFA5B8A9AE
:106840001D921D921D921C921397810101591E4F9A
:10685000F80180818823E9F1E259FE4F608171815E
:10686000072E000C880B990B0E942E4F9B01AC0148
:10687000F101E954FD4F60817181828193810E9411
:10688000B551181634F5D8011C926FED73E005551B
:106890001F4FC8010E94EE2A64E775E0C8010E94FC
:1068A000EE2A6CE877E0C8010E94EE2A6396BFAD3D
:1068B0006397BB2309F4D8C0F101E651FE4F108A5B
:1068C000118A128A138AE9A9FAA910821182128206
:1068D000138260E0C2010E94190D882369F0F10162
:1068E000E25BFF4F1082118212821382E45CFE4F42
:1068F000108A118A128A138A60E0C3010E94190D5E
:10690000882371F0AFA5B8A91D921D921D921C920B
:106910001397F101E654FE4F108A118A128A138AE6
:1069200060E0C4010E94190D882369F0E9A9FAA961
:106930001082118212821382F101E651FE4F108AF9
:10694000118A128A138AF101ED58FF4F8081AB89B9
:10695000BC898C93E258FF4F8081EB8DFC8D808346
:10696000F101E159FE4F8081ABA1BCA18C93E152B2
:10697000F14020813181428153812FA338A749A75B
:106980005AA7AFA5B8A98D919D910D90BC91A02D4E
:106990008F839887A987BA87E9A9FAA9C080D1808F
:1069A000E280F3800E942A122FA138A549A55AA59A
:1069B0002093DC083093DD084093DE085093DF0815
:1069C0000E942A128F819885A985BA858093E00854
:1069D0009093E108A093E208B093E3080E942A1282
:1069E000C092E408D092E508E092E608F092E70849
:1069F0000E94B312AB89BC898C91882309F46AC0C8
:106A00000E94250A2B853C854D855E85621773079C
:106A10008407950768F50E94250A2B853C854D85DE
:106A20005E85621773078407950708F053C00E94BC
:106A3000250A6B017C01F101E956FD4F208131816E
:106A400042815381A8EEB3E00E9476506C157D051B
:106A50008E059F0550F13EC073E0A72EB12CAECE3F
:106A600063E0A62EB12CF1CE53E0A52EB12C31CF90
:106A70000E94250A6B017C012B853C854D855E8536
:106A8000C21AD30AE40AF50AF101E956FD4F208142
:106A9000318142815381A8EEB3E00E9476506C159B
:106AA0007D058E059F0508F0B6CF62E472E0810196
:106AB000065E1D4FC8010E94EE2A6CE877E0C8010F
:106AC0000E94EE2A6CE975E0C8010E94EE2A42E0BD
:106AD000A42EB12CAB8DBC8D8C91882309F45DC0A4
:106AE0000E94250A2B853C854D855E8562177307BC
:106AF0008407950708F50E94250A2B853C854D855E
:106B00005E85621773078407950708F046C00E94E8
:106B1000250A6B017C01F101E556FD4F2081318191
:106B200042815381A8EEB3E00E9476506C157D053A
:106B30008E059F05E8F031C00E94250A6B017C019B
:106B40002B853C854D855E85C21AD30AE40AF50A79
:106B5000F101E556FD4F2081318142815381A8EE3C
:106B6000B3E00E9476506C157D058E059F0518F6E2
:106B70006EE372E08101065E1D4FC8010E94EE2A9D
:106B80006CE877E0C8010E94EE2A61EB75E0C8016D
:106B90000E94EE2A32E0A32EB12CABA1BCA18C91B5
:106BA000882309F45DC00E94250A2B853C854D850C
:106BB0005E85621773078407950708F50E94250A0A
:106BC0002B853C854D855E85621773078407950785
:106BD00008F046C00E94250A6B017C01F101E156D4
:106BE000FD4F2081318142815381A8EEB3E00E94A4
:106BF00076506C157D058E059F05E8F031C00E942A
:106C0000250A6B017C012B853C854D855E85C21A6A
:106C1000D30AE40AF50AF101E156FD4F20813181E2
:106C200042815381A8EEB3E00E9476506C157D0539
:106C30008E059F0518F66AE372E08101065E1D4F1E
:106C4000C8010E94EE2A6CE877E0C8010E94EE2A93
:106C500066EC75E0C8010E94EE2A22E0A22EB12C5B
:106C60008EE79CE00E94F607181619060CF040C04B
:106C70008EE79CE00E94D4078F7D85349105C1F595
:106C800064EB74E0C101865E9D4F0E94EE2A86E5AA
:106C900092E00E94D9130E942A120E940F14F1015F
:106CA000ED58FF4F1082E258FF4F1082E258FF4F1D
:106CB0001082AB89BC891C92EB8DFC8D1082ABA13C
:106CC000BCA11C92B1E0BF87AA24A394B12C6BEDA8
:106CD00075E0C101865E9D4F0E94EE2AEB89FC891A
:106CE0001082AB8DBC8D1C92EBA1FCA1108203C065
:106CF000A114B10461F7C1010E944D27F101EA5DC1
:106D0000FD4F808191810196918380838D329140E6
:106D10000CF456CCD101A25EBD4F8D919C91119780
:106D2000892B09F04DCC14968D919C91892B09F0FB
:106D300047CC118210823297808191810097A1F017
:106D4000019759F1F101EC5DFD4F80819181019630
:106D5000823091050CF0EBC091838083F101EE5DF0
:106D6000FD4F118210822CCC62E572E08101065E3B
:106D70001D4FC8010E94EE2A0E942A12CE010196E0
:106D80000E94F72ABE016F5F7F4FC8010E94402B0F
:106D9000CE0101960E94CA26D5CF0E942A128C01EC
:106DA000FC0180819181A281B381181619061A060F
:106DB0001B0644F081E090E0A0E0B0E08083918386
:106DC000A283B383F80184819581A681B7811816C7
:106DD00019061A061B0644F081E090E0A0E0B0E03E
:106DE00084839583A683B783F80180859185A285E6
:106DF000B385181619061A061B0644F081E090E0C8
:106E0000A0E0B0E080879187A287B3871A821982B9
:106E10001C821B821E821D8270E060E0CE01019602
:106E20000E94282760E274E0CE0101960E94EE2ABB
:106E300065E374E0CE0101960E94EE2A6091DC08C1
:106E40007091DD088091DE089091DF080E942E4F3E
:106E50006B017C01D8016D917D918D919C910E9477
:106E60002E4F9B01AC01C701B6010E941C51AB0122
:106E7000BC01CE0101960E94BE2A65E474E0CE01F9
:106E800001960E94EE2A6091E0087091E1088091DD
:106E9000E2089091E3080E942E4F6B017C01F801FB
:106EA00064817581868197810E942E4F9B01AC0180
:106EB000C701B6010E941C51AB01BC01CE01019675
:106EC0000E94BE2A65E574E0CE0101960E94EE2A7A
:106ED0006091E4087091E5088091E6089091E708D8
:106EE0000E942E4F6B017C01D80118966D917D9107
:106EF0008D919C911B970E942E4F9B01AC01C70165
:106F0000B6010E941C51AB01BC01CE0101960E944A
:106F1000BE2ABE016F5F7F4F8101065E1D4FC80113
:106F20000E94402BCE0101960E94CA2625CF1182D5
:106F3000108214CF87EE95E00E94D9136196FFADC1
:106F40006197FF2379F1A114B104B9F52F852111BF
:106F500034C086E392E00E94D9130E942A120E9454
:106F60000F1462963FAD6297332341F082E392E0C3
:106F70000E94D9130E942A120E940F1463968FADAB
:106F800063978823D1F0A114B104B9F49F859111BE
:106F900014C08EE292E00E94D9130E942A120E942D
:106FA0000F140BC062965FAD6297552339F3A1149D
:106FB000B10419F44F854423C9F285E090E0ABA5F4
:106FC000BCA58D939C938101035D1D4FF8019183B6
:106FD00080839101215D3D4F3C872B87D9018D93A3
:106FE0009C9345E050E0B201C1010E94462BF8019C
:106FF00040815181B301C1010E94462BAB85BC8504
:107000004D915C91B401C1010E94462BC1010E94C7
:10701000FA11F101E25BFF4F2081318142815381FE
:107020002F8F38A349A35AA3E258FF4F8081918143
:10703000A281B3818F8B988FA98FBA8FE258FF4FAF
:10704000C080D180E280F3800E942A122F8D38A167
:1070500049A15AA12093DC083093DD084093DE0853
:107060005093DF080E942A128F89988DA98DBA8DBE
:107070008093E0089093E108A093E208B093E308BE
:107080000E942A12C092E408D092E508E092E60835
:10709000F092E7080E94B3120E9415150E942A126E
:1070A0000E94EC18C1010E948C19ABA5BCA51D92D1
:1070B0001C92F80111821082AB85BC851D921C9236
:1070C00050E040E0B201C1010E94462BF80140812E
:1070D0005181B301C1010E94462BAB85BC854D9106
:1070E0005C91B401C1010E94462BC1010E94FA11BA
:1070F000BF85BB2341F00E942A1221E0FC012687B4
:10710000AA24A394B12C85EF95E00E94D913C50160
:107110000E940A148CE897E00E94D9130E942A1258
:10712000B0920C08A0920B08C501E8960FB6F8942F
:10713000DEBF0FBECDBFDF91CF911F910F91FF90AA
:10714000EF90DF90CF90BF90AF909F908F907F9007
:107150006F905F904F903F902F9008958F929F92E5
:10716000AF92BF92CF92DF92EF92FF920F931F9355
:107170000E94BA2962E070E00E94942B892BD1F41E
:107180000E94BA2921E02F931F921F921F921F92F3
:10719000912C812CB12CA12CC12CD12C76019701E2
:1071A0008601B701A6010E945A300F900F900F90F0
:1071B0000F900F9090E080E01F910F91FF90EF9063
:1071C000DF90CF90BF90AF909F908F9008952F92B7
:1071D0003F924F925F926F927F928F929F92AF9267
:1071E000BF92CF92DF92EF92FF920F931F93CF93B4
:1071F000DF930E94001B8091C2099091C3090197FF
:1072000009F055C086EF9FEFD0E0C0E02C01990F48
:1072100066087708C330D10509F44CC0C530D105E4
:1072200009F448C0C130D10509F444C00E94BA290C
:107230001F9221E02F931F921F921F92912C812C5D
:10724000B12CA12CC12CD12C760197018601B7015C
:10725000A6010E945A300F900F900F900F900F9040
:107260000E942A1220900B0830900C080E942A12CB
:10727000FC018685811106C0232821F42196C730A0
:10728000D10541F690E080E0DF91CF911F910F9101
:10729000FF90EF90DF90CF90BF90AF909F908F9036
:1072A0007F906F905F904F903F902F9008958AE06D
:1072B00090E0AACF0E94BA291C01C301B2010E942A
:1072C0002E4F8B019C011F921F921F921F921F92A3
:1072D000912C812CB12CA12CC12CD12C7601B70181
:1072E000A601C101B6CF4F925F926F927F928F92AB
:1072F0009F92AF92BF92CF92DF92EF92FF920F9345
:107300001F93CF93DF9300D01F92CDB7DEB70E94BB
:10731000001B4090D2095090D3096090D40970901E
:10732000D5090E94001B8090D6099090D709A090A3
:10733000D809B090D9090E942A12C090DC08D090D8
:10734000DD08E090DE08F090DF080E942A12C701F5
:10735000B6010E942E4F6B017C01C301B2010E9455
:107360002E4F9B01AC01C701B6010E941C512B019D
:107370003C016091E0087091E1088091E2089091F1
:10738000E3080E942E4F6B017C01C501B4010E94ED
:107390002E4F9B01AC01C701B6010E941C516983AD
:1073A0007A838B839C830E94BA291F921F921F921B
:1073B0001F921F92912C812CB12CA12CC12CD12C6D
:1073C000760109811A812B813C81B301A2010E94BF
:1073D0005A300E94BA291F921F921F921F921F9229
:1073E00097018601B301A2010E945A300E94BA2976
:1073F0001F921F921F921F921F929701B701A60121
:107400000E945A300FB6F894DEBF0FBECDBF90E099
:1074100080E00F900F900F900F90DF91CF911F9110
:107420000F91FF90EF90DF90CF90BF90AF909F9023
:107430008F907F906F905F904F9008952F923F9222
:107440004F925F926F927F928F929F92AF92BF9274
:10745000CF92DF92EF92FF920F931F93CF93DF9320
:107460000E94001B8091C2099091C309019709F005
:1074700055C086EF9FEFD0E0C0E02C01990F660861
:107480007708C330D10509F44CC0C530D10509F4E3
:1074900048C0C130D10509F444C00E94BA291F92E6
:1074A0001F9221E02F931F921F92912C812CB12CBF
:1074B000A12CC12CD12C760197018601B701A60120
:1074C0000E945A300F900F900F900F900F900E94D3
:1074D0002A1220900B0830900C080E942A12FC01FE
:1074E0008685811106C0232821F42196C730D10555
:1074F00041F690E080E0DF91CF911F910F91FF90D6
:10750000EF90DF90CF90BF90AF909F908F907F9043
:107510006F905F904F903F902F9008958AE090E099
:10752000AACF0E94BA291C01C301B2010E942E4FAA
:10753000AB01BC011F921F921F921F921F92912CB0
:10754000812CB12CA12CC12CD12C76019701860164
:10755000C101B6CF8F929F92AF92BF92CF92DF922E
:10756000EF92FF920F931F93CF93DF93EB010E9453
:10757000BA298A889B88AE84BF84CA84DB84EC8461
:10758000FD840E811F81288539854A815B816C814C
:107590007D811F921F921F92EF89EF93EE89EF93E7
:1075A0000E945A300F900F900F900F900F9090E024
:1075B00080E0DF91CF911F910F91FF90EF90DF90CE
:1075C000CF90BF90AF909F908F9008952F923F9251
:1075D0004F925F926F927F928F929F92AF92BF92E3
:1075E000CF92DF92EF92FF920F931F93CF93DF938F
:1075F0000E94BA2921E02F931F921F921F921F927F
:10760000912C812CB12CA12CC12CD12C760197016D
:107610008601B701A6010E945A300E94001B0F90FC
:107620000F900F900F900F908091C2099091C30915
:10763000019709F055C086EF9FEFD0E0C0E02C0124
:10764000990F66087708C330D10509F44CC0C530DE
:10765000D10509F448C0C130D10509F444C00E94E5
:10766000BA2921E02F931F921F921F921F92912CF3
:10767000812CB12CA12CC12CD12C76019701860133
:10768000B701A6010E945A300F900F900F900F90F3
:107690000F900E942A1220900B0830900C080E9434
:1076A0002A12FC018685811106C0232821F4219627
:1076B000C730D10541F690E080E0DF91CF911F9176
:1076C0000F91FF90EF90DF90CF90BF90AF909F9081
:1076D0008F907F906F905F904F903F902F90089584
:1076E0008AE090E0AACF0E94BA291C01C301B2012E
:1076F0000E942E4F6B017C011F921F921F921F92BE
:107700001F92912C812CB12CA12C00E010E098014B
:10771000B901A801C101B6CF8F929F92AF92BF92DB
:10772000CF92DF92EF92FF920F931F930E94BA299C
:1077300070E060E00E94942B892BD1F40E94BA295A
:107740001F921F9221E02F931F921F92912C812C48
:10775000B12CA12CC12CD12C760197018601B70147
:10776000A6010E945A300F900F900F900F900F902B
:1077700090E080E01F910F91FF90EF90DF90CF900D
:10778000BF90AF909F908F9008958F929F92AF92ED
:10779000BF92CF92DF92EF92FF920F931F930E94BE
:1077A000BA2961E070E00E94942B892BD1F40E94E9
:1077B000BA291F9221E02F931F921F921F92912CA2
:1077C000812CB12CA12CC12CD12C760197018601E2
:1077D000B701A6010E945A300F900F900F900F90A2
:1077E0000F9090E080E01F910F91FF90EF90DF905D
:1077F000CF90BF90AF909F908F9008951F920F925F
:107800000FB60F9211240BB60F922F933F934F9305
:107810005F936F937F938F939F93AF93BF93EF93F8
:10782000FF938EE79CE00E940B08FF91EF91BF91C0
:10783000AF919F918F917F916F915F914F913F9108
:107840002F910F900BBE0F900FBE0F901F901895A9
:107850001F920F920FB60F9211240BB60F922F9317
:107860008F939F93EF93FF93E0918E0CF0918F0C89
:107870008081E091940CF091950C82FD1DC0908167
:107880008091970C8F5F8F732091980C821741F035
:10789000E091970CF0E0E258F34F958F8093970CAE
:1078A000FF91EF919F918F912F910F900BBE0F90B1
:1078B0000FBE0F901F9018958081F2CF1F920F92EC
:1078C0000FB60F9211242F933F938F939F93AF93F3
:1078D000BF938091D2079091D307A091D407B09124
:1078E000D5073091D10723E0230F2D3758F50196A6
:1078F000A11DB11D2093D1078093D2079093D30788
:10790000A093D407B093D5078091D6079091D7075D
:10791000A091D807B091D9070196A11DB11D809300
:10792000D6079093D707A093D807B093D907BF91F4
:10793000AF919F918F913F912F910F900FBE0F901C
:107940001F90189526E8230F0296A11DB11DD2CFD6
:107950001F920F920FB60F9211240BB60F922F9316
:107960003F934F935F936F937F938F939F93AF93C7
:10797000BF93EF93FF9348E251E064E271E090E03F
:1079800080E00E94340BFF91EF91BF91AF919F91E6
:107990008F917F916F915F914F913F912F910F90B8
:1079A0000BBE0F900FBE0F901F9018951F920F9255
:1079B0000FB60F9211240BB60F922F933F934F9354
:1079C0005F936F937F938F939F93AF93BF93EF9347
:1079D000FF9348EA50E064EA70E083E090E00E94A0
:1079E000340BFF91EF91BF91AF919F918F917F9158
:1079F0006F915F914F913F912F910F900BBE0F9020
:107A00000FBE0F901F9018951F920F920FB60F92F6
:107A100011240BB60F922F933F934F935F936F9365
:107A20007F938F939F93AF93BF93EF93FF9348E917
:107A300050E064E970E082E090E00E94340BFF9136
:107A4000EF91BF91AF919F918F917F916F915F91D6
:107A50004F913F912F910F900BBE0F900FBE0F9043
:107A60001F9018951F920F920FB60F9211240BB60C
:107A70000F922F933F934F935F936F937F938F93C7
:107A80009F93AF93BF93EF93FF9348E850E064E870
:107A900070E081E090E00E94340BFF91EF91BF9184
:107AA000AF919F918F917F916F915F914F913F9196
:107AB0002F910F900BBE0F900FBE0F901F90189537
:107AC0001F920F920FB60F9211240BB60F922F93A5
:107AD0003F934F935F936F937F938F939F93AF9356
:107AE000BF93EF93FF93E091DB07F091DC071995CB
:107AF000FF91EF91BF91AF919F918F917F916F9186
:107B00005F914F913F912F910F900BBE0F900FBE41
:107B10000F901F9018951092810C1092800C88EE97
:107B200093E0A0E0B0E08093820C9093830CA0934C
:107B3000840CB093850C82E793E090937F0C809344
:107B40007E0C85EC90E090938B0C80938A0C84ECF7
:107B500090E090938D0C80938C0C80EC90E090934F
:107B60008F0C80938E0C81EC90E09093910C80931D
:107B7000900C82EC90E09093930C8093920C86ECA6
:107B800090E09093950C8093940C1092970C109227
:107B9000980C1092990C10929A0CECEAFDE02FEFE1
:107BA00048EB5BE08091AB0D803320F591E0980FBE
:107BB0009093AB0D808390E0DC01AA0FBB1FA80F50
:107BC000B91FA55EB24F12965C934E9311973396F0
:107BD0008DE0E83BF80731F782E090E00E94AF4982
:107BE00024E833E0FC01318320839093B90D809326
:107BF000B80D08952083EBCF789484B5826084BD5E
:107C000084B5816084BD85B5826085BD85B58160A0
:107C100085BD80916E00816080936E00109281001E
:107C200080918100826080938100809181008160D9
:107C3000809381008091800081608093800080919A
:107C4000B10084608093B1008091B0008160809326
:107C5000B0008091910082608093910080919100AA
:107C6000816080939100809190008160809390006A
:107C70008091A10082608093A1008091A100816029
:107C80008093A1008091A00081608093A0008091EA
:107C90002101826080932101809121018160809384
:107CA00021018091200181608093200180917A00E0
:107CB000846080937A0080917A00826080937A0059
:107CC00080917A00816080937A0080917A00806848
:107CD00080937A001092C100E0918E0CF0918F0C8D
:107CE00082E08083E0918A0CF0918B0C1082E0910D
:107CF0008C0CF0918D0CD0E1D0831092960CE09119
:107D0000920CF091930C86E08083E091900CF091BE
:107D1000910C808180618083E091900CF091910CB6
:107D2000808188608083E091900CF091910C80813B
:107D300080688083E091900CF091910C80818F7D20
:107D4000808364E670E080E090E00E94F4098FE5B3
:107D500092E00E94D9138DE592E00E94D91380E051
:107D600096E00E94D9138AE592E00E94D91361E05F
:107D700086E30E94880961E087E30E94880961E048
:107D800086E20E94880961E08AE10E94880961E038
:107D90008CE10E94880961E088E10E94880962E024
:107DA00083E00E94880962E082E00E94880962E024
:107DB00080E10E94880962E081E10E94880962E016
:107DC0008FE10E94880962E081E20E94880961E0F7
:107DD0008CE30E94880961E08DE30E94880961E0DC
:107DE00088E30E94880962E08EE00E94880962E0D0
:107DF0008FE00E94880962E087E10E94880962E0C2
:107E000089E10E94880962E083E20E94880962E0B9
:107E100085E20E94880961E08EE20E94880961E0A3
:107E200080E30E94880961E08EE30E94880962E095
:107E300082E10E94880962E083E10E94880962E091
:107E40008BE10E94880962E08DE10E94880962E06E
:107E500087E20E94880962E089E20E94880961E065
:107E60008AE00E94880961E088E00E94880961E058
:107E700089E00E94880961E08DE00E94880960E045
:107E80008AE00E945B0960E088E00E945B0960E094
:107E900089E00E945B0960E08DE00E945B0962E07E
:107EA0008FE30E94880962E08BE30E94880962E008
:107EB00088E20E94880962E080E40E94880962E00A
:107EC0008AE20E94880962E08CE20E94880962E0EE
:107ED00081E40E94880962E082E40E94880962E0ED
:107EE00084E30E94880962E085E30E94880962E0D9
:107EF00080E00E94880962E081E00E94880962E0D7
:107F000089E30E94880962E08AE30E94880962E0AE
:107F100081E30E94880962E082E30E94880962E0AE
:107F200083E30E94880962E08BE20E94880962E094
:107F30008DE20E94880962E08FE20E94880962E077
:107F400080E20E94880961E084E00E94880961E083
:107F500085E00E94880961E086E00E94880961E06E
:107F60008BE00E94880960E084E00E945B0960E089
:107F700085E00E945B0960E086E00E945B0960E0AA
:107F80008BE00E945B098FE592E00E94D9138DE59A
:107F900092E00E94D9138AE196E00E94D9138AE503
:107FA00092E00E94D9138FE592E00E94D9138DE5EB
:107FB00092E00E94D9138BE296E00E94D9138AE5E1
:107FC00092E00E94D9130E94001B0E947E158FE54B
:107FD00092E00E94D9138DE592E00E94D9138BE3C1
:107FE00096E00E94D9138AE592E00E94D9130E947C
:107FF000BA290E9432258FE592E00E94D9138DE5BF
:1080000092E00E94D91382E596E00E94D9138AE596
:1080100092E00E94D91361E086E20E945B0961E070
:1080200088E10E945B0961E088E30E945B0961E0EE
:108030008EE30E945B098FE592E00E94D9138DE5E3
:1080400092E00E94D91388E696E00E94D9138AE54F
:1080500092E00E94D9130E94F91B0E94C91B0E9442
:10806000250A0E94250A6093DD077093DE0780933E
:10807000DF079093E0078FE592E00E94D9138DE52A
:1080800092E00E94D91388E796E00E94D9138AE50E
:1080900092E00E94D9130E94BB1264E070E08CEA67
:1080A0009DE00E94AD0A65E070E08FEA9DE00E94CD
:1080B000AD0A66E070E082EB9DE00E94AD0A6BE0E5
:1080C00070E085EB9DE00E94AD0A8FE592E00E9492
:1080D000D9138DE592E00E94D91384E896E00E94BE
:1080E000D9138AE592E00E94D91383ED99E2909327
:1080F000DC078093DB07C1E0C0936F00D093810061
:1081000010928000C093DA0780E092E0909387009D
:108110008093860081E1809381001092810010920B
:108120008500109284008091DA078061809381003D
:108130000E94250A6093EC087093ED088093EE0886
:108140009093EF088FE592E00E94D9138DE592E0BD
:108150000E94D91384E996E00E94D9138AE592E03F
:108160000E94D9130E94001B8091FE089091FF0885
:10817000A0910009B09101090197A105B10559F538
:108180000E94001B8091460990914709A0914809DF
:10819000B09149090197A105B105E9F489EA96E092
:1081A0000E94D9130E94BA29CF931F921F921F9247
:1081B0001F92912C812CB12CA12CC12CD12C760199
:1081C00097018601B701A6010E945A300F900F90C7
:1081D0000F900F900F900E94001B8091FE089091CD
:1081E000FF08A0910009B09101090197A105B1050F
:1081F00061F50E94001B8091420990914309A09172
:108200004409B09145090197A105B105F1F481EC4C
:1082100096E00E94D9130E94BA291F9221E02F9361
:108220001F921F921F92912C812CB12CA12CC12C3A
:10823000D12C760197018601B701A6010E945A3020
:108240000F900F900F900F900F900E94001B809145
:10825000FE089091FF08A0910009B09101090197D3
:10826000A105B10561F50E94001B80913E09909126
:108270003F09A0914009B09141090197A105B105BD
:10828000F1F489ED96E00E94D9130E94BA291F9259
:108290001F9221E02F931F921F92912C812CB12CC1
:1082A000A12CC12CD12C760197018601B701A60122
:1082B0000E945A300F900F900F900F900F9088E609
:1082C00092E00E94D91386E692E00E94D91381EFD2
:1082D00096E00E94D91383E692E00E94D913EEE063
:1082E0006E2E712CFEED2F2EF2E03F2E0E94250AFD
:1082F000AB01BC018091DD079091DE07A091DF0703
:10830000B091E007481759076A077B0708F060C07B
:108310004093DD075093DE076093DF077093E0071B
:108320008EE79CE00E94F607892B09F424C30E9483
:10833000250A6093EC087093ED088093EE08909303
:10834000EF088EE79CE00E94D4078093D808982F0E
:108350009F7D953409F468C02091D6083091D708E4
:10836000F901EE58F74F80832F5F3F4F3093D708C6
:108370002093D6088091D6089091D708833691052E
:1083800064F02AE02093D808FC01EE58F74F2083D0
:1083900001969093D7088093D6082091D608309103
:1083A000D7088091D8088A3021F0243631050CF4A2
:1083B000E2C2C9010197ADE0B8E0E2E7F8E0AF0141
:1083C0004257584048175907B4F541914D93F7CF9C
:1083D000481B590B6A0B7B0B483E534061057105E6
:1083E00008F49ECF88519C4FAF4FBF4F8093DD075D
:1083F0009093DE07A093DF07B093E0070E94F91B7C
:10840000EC010E949814CE010C960E949814CE01A3
:1084100048960E949814CE0184960E949814CE012A
:10842000C0960E9498147CCF0E942A1221E0DC01A1
:108430001E962C939FCF835F974FFC0110822230B2
:1084400031050CF494C28AE593E00E94D91387EBBE
:1084500093E00E94D9138AE097E00E94D9138DE03F
:1084600098E00E94D9138AE097E00E94D9138CE823
:1084700097E00E94D9138AE390E071D7EC011A8249
:108480001B821C821D821E821F82188619861A86F4
:108490001B861C861D861E861F86188A198A1A8AC4
:1084A0001B8A1C8A1D8A1E8A1F8A188E198E1A8E94
:1084B0001B8E1C8E1D8E1E8E1F8E18A219A21AA234
:1084C0001BA21CA21DA21EA21FA218A619A61AA6B4
:1084D0001BA61CA61DA61EA61FA618AA19AA1AAA84
:1084E0001BAA1CAA1DAA1EAA1FAA18AE19AE6DE1CE
:1084F00072E08DE098E00E94D74A8C01DC018C91FB
:108500008654823008F0DFC16CE077E0C8010E9439
:10851000C852892B09F48FC16FE077E0C8010E942F
:10852000C852892B09F487C163E177E0C8010E9432
:10853000C852892B09F482C166E177E0C8010E9424
:10854000C852892B09F47AC16AE177E0C8010E9418
:10855000C852892B09F475C16EE177E0C8010E9409
:10856000C852892B09F470C162E277E0C8010E9409
:10857000C852892B09F468C165E277E0C8010E94FE
:10858000C852892B09F463C169E277E0C8010E94EF
:10859000C852892B09F45EC16DE277E0C8010E94E0
:1085A000C852892B09F459C161E377E0C8010E94E0
:1085B000C852892B09F454C165E377E0C8010E94D1
:1085C000C852892B09F44FC169E377E0C8010E94C2
:1085D000C852892B09F44AC16DE377E0C8010E94B3
:1085E000C852892B09F445C161E477E0C8010E94B3
:1085F000C852892B09F440C165E477E0C8010E94A4
:10860000C852892B09F43BC169E477E0C8010E9494
:10861000C852892B09F436C16DE477E0C8010E9485
:10862000C852892B09F431C161E577E0C8010E9485
:10863000C852892B09F42CC165E577E0C8010E9476
:10864000C852892B09F427C169E577E0C8010E9467
:10865000C852892B09F422C16DE577E0C8010E9458
:10866000C852892B09F41DC161E677E0C8010E9458
:10867000C852892B09F418C165E677E0C8010E9449
:10868000C852892B09F413C169E677E0C8010E943A
:10869000C852892B09F40EC16DE677E0C8010E942B
:1086A000C852892B09F409C161E777E0C8010E942B
:1086B000C852892B09F004C188EB90E09093010225
:1086C000809300020115110509F403C1F8018081AE
:1086D000883539F4C801019667D76A837B838C8318
:1086E0009D83D8018C91893539F4C80101965CD7F6
:1086F0006E837F8388879987F80180818A3539F472
:10870000C801019651D76A877B878C879D87D801DE
:108710008C91813449F4C801019646D70E94845156
:108720006E877F87888B998BF8018081823449F42A
:10873000C801019639D70E9484516A8B7B8B8C8B40
:108740009D8BD8018C91833449F4C80101962CD7B4
:108750000E9484516E8B7F8B888F998FF801808166
:10876000833539F4C80101961FD76A8F7B8F8C8FB0
:108770009D8FD8018C91803549F4C801019614D79A
:108780000E9484516E8F7F8F88A399A3F801808106
:10879000863549F4C801019607D70E9484516AA31F
:1087A0007BA38CA39DA3D8018C91873549F4C80184
:1087B0000196FAD60E9484516EA37FA388A799A739
:1087C000F8018081853449F4C8010196EDD60E94F4
:1087D00084516AA77BA78CA79DA7D8018C9184356B
:1087E00049F4C8010196E0D60E9484516EA77FA784
:1087F00088AB99ABF80180818D3449F4C8010196AA
:10880000D3D60E9484516AAB7BAB8CAB9DABD801B5
:108810008C91813549F4C8010196C6D60E948451D5
:108820006EAB7FAB88AF99AF65E777E090E080E013
:10883000BED68C0147CF90E080E040CF81E090E051
:108840003DCF8CE190E03ACF8DE690E037CF8FE6D8
:1088500090E034CF80E790E031CF81E790E02ECFF9
:1088600082E790E02BCF83E790E028CF84E790E089
:1088700025CF88E790E022CF89E790E01FCF8AE7F5
:1088800090E01CCF83E890E019CF84E890E016CF09
:108890008DE890E013CF8EE890E010CF8FE890E065
:1088A0000DCF80E990E00ACF81EA90E007CF85EB19
:1088B00090E004CF86EB90E001CF87EB90E0FECE16
:1088C0008FEF9FEFFBCE8FEF9FEF9093010280938E
:1088D00000020E942A12FC0116850E94001B809053
:1088E0000A0990900B09A0900C09B0900D09CEA830
:1088F000DFA8E8ACF9AC0E942A12C0927A0CD092A0
:108900007B0CE0927C0CF0927D0C809100029091A7
:1089100001028230910508F4DEC49C012F56310912
:108920002530310508F4D7C4552453948437910574
:1089300009F0512C112309F4D2C48D36910509F4A4
:10894000CEC49C01285731092330310508F4C7C42F
:10895000855B9109039708F4C2C486E593E00E9401
:10896000D9130E942A120E940F14CE0194D510929E
:10897000D7081092D6088091D9088111A4C00E940E
:108980002A12FC018685882309F49DC00E94BA2919
:10899000EC01FC01E05FFC4F108240960E947C0CD1
:1089A000CE0182579F4F0E947C0CCE01845F9E4F68
:1089B0000E947C0C0E9415138C010F5F1F4FC1E0B9
:1089C000D0E0D8018D918D018823D9F08FED93E00F
:1089D0000E94D9138FE897E00E94D913CE010E941C
:1089E0000A148CE897E00E94D91360E08C2F0E9453
:1089F0005B0970E060E0CE010E943614F801319707
:108A00001082F80187A98823F9F08FED93E00E9486
:108A1000D91386EA97E00E94D913CE010E940A1466
:108A20008CE897E00E94D91361E08C2F0E9488099E
:108A300060E08C2F0E945B0961E070E0CE010E9433
:108A40003614D801D7961C922196C533D10509F06A
:108A5000B8CF0E94BB122091AC0D30E0C901880F45
:108A6000991F820F931FFC01E55EF24F80818F7B7F
:108A700080832091AF0D30E0C901880F991F820FCC
:108A8000931FFC01E55EF24F80818F7B80832091F4
:108A9000B20D30E0C901880F991F820F931FFC01AE
:108AA000E55EF24F80818F7B80832091B50D30E0B1
:108AB000C901880F991F820F931FFC01E55EF24FD9
:108AC00080818F7B80830E942A12FC01868580939F
:108AD000D9080E94001B2091DA083091DB08DC01E4
:108AE00012968D919C912817390789F00E94001BDE
:108AF000FC01828193819093DB088093DA080E94C5
:108B0000BA290E9432250E94F91B0E94C91B0E94AB
:108B1000250A0091EC081091ED082091EE083091A3
:108B2000EF08601771078207930708F0F0C20E94F0
:108B3000250A6093EC087093ED088093EE089093FB
:108B4000EF080E949C08D2CB209779F48EE493E042
:108B50000E94D9130E942A120E940F140E942A1206
:108B600070920C0860920B0800CFE0900002F09029
:108B70000102FFEFEF16FF0649F3E114F10409F0DB
:108B800083C08091090890910A08892B61F482E0E2
:108B900090E0E5D328E333E0DC012D933C93909300
:108BA0000A08809309080091090810910A08B1E7A2
:108BB000EB16F10409F09EC08091FF079091000828
:108BC000892B61F482E090E0CAD326E033E0FC0117
:108BD00031832083909300088093FF070091FF0763
:108BE00010910008F9E7EF16F10409F09EC080919A
:108BF000F5079091F607892B61F482E090E0AFD3FE
:108C0000E4EDF2E0DC01ED93FC939093F6078093A2
:108C1000F5070091F5071091F607F0E9EF16F1045A
:108C200009F09EC08091EB079091EC07892B61F4CD
:108C300082E090E094D3E2EAF2E0DC01ED93FC9371
:108C40009093EC078093EB070091EB071091EC07F2
:108C5000F8EBEF16F10409F09EC08091E1079091C6
:108C6000E207892B61F482E090E079D3E0E7F2E05B
:108C7000DC01ED93FC939093E2078093E107009170
:108C8000E1071091E20787C0BCE1EB16F104B9F4EB
:108C90008091070890910808892B61F482E090E0A8
:108CA0005ED32EE233E0FC013183208390930808E9
:108CB00080930708009107081091080878CFFDE617
:108CC000EF16F10409F082C0809105089091060822
:108CD000892B61F482E090E042D324E233E0DC01AE
:108CE0002D933C9390930608809305080091050806
:108CF00010910608F2E7EF16F10409F082C08091A6
:108D0000FD079091FE07892B61F482E090E027D364
:108D10002CEF32E0DC012D933C939093FE0780937F
:108D2000FD070091FD071091FE07FAE7EF16F10429
:108D300009F082C08091F3079091F407892B61F4C8
:108D400082E090E00CD3EAECF2E0DC01ED93FC93DE
:108D50009093F4078093F3070091F3071091F407C1
:108D6000F1EAEF16F10409F082C08091E9079091D1
:108D7000EA07892B61F482E090E0F1D2E8E9F2E0C1
:108D8000DC01ED93FC939093EA078093E90700914F
:108D9000E9071091EA070115110509F044C18EE4B5
:108DA00093E00E94D9130E942A120E940F140E947D
:108DB0002A1270920C0860920B0889E797E00E94D3
:108DC00089138CE897E00E948913CFCDBFE6EB169C
:108DD000F10409F068C08091030890910408892B80
:108DE00061F482E090E0BBD22AE133E0FC01318300
:108DF0002083909304088093030800910308109146
:108E00000408B3E7EB16F10409F0BBC08091FB073F
:108E10009091FC07892B61F482E090E0A0D222EFD0
:108E200032E0FC01318320839093FC078093FB07A1
:108E30000091FB071091FC07FDE8EF16F10409F023
:108E4000BBC08091F1079091F207892B61F482E019
:108E500090E085D2E0ECF2E0DC01ED93FC9390939E
:108E6000F2078093F1070091F1071091F207F5EBFB
:108E7000EF16F10409F0BBC08091E7079091E80775
:108E8000892B61F482E090E06AD2EEE8F2E0DC0146
:108E9000ED93FC939093E8078093E7070091E70731
:108EA0001091E80778CFF0E7EF16F10409F066C0FB
:108EB0008091010890910208892B61F482E090E092
:108EC0004ED220E133E0DC012D933C9390930208D5
:108ED000809301080091010810910208B8E7EB1691
:108EE000F10409F07FCE8091F7079091F807892B64
:108EF00051F482E090E033D2FC01318220829093E1
:108F0000F8078093F7070091F7071091F807FFE83B
:108F1000EF16F10409F081CE8091ED079091EE07F4
:108F2000892B61F482E090E01AD2ECEAF2E0DC01F5
:108F3000ED93FC939093EE078093ED070091ED077E
:108F40001091EE07F7EBEF16F10409F081CE809156
:108F5000E3079091E407892B61F482E090E0FFD170
:108F6000EAE7F2E0DC01ED93FC939093E407809351
:108F7000E3070091E3071091E4070DCF10E000E054
:108F800016CEF4E7EF16F10409F0A8CF8091F907A7
:108F90009091FA07892B61F482E090E0E0D128EE0D
:108FA00032E0DC012D933C939093FA078093F9070C
:108FB0000091F9071091FA07FEE8EF16F10409F0A5
:108FC000A6CF8091EF079091F007892B61F482E0A2
:108FD00090E0C5D1E6EBF2E0DC01ED93FC939093D9
:108FE000F0078093EF070091EF071091F007F6EB81
:108FF000EF16F10409F0A6CF8091E5079091E607FE
:10900000892B61F482E090E0AAD1E4E8F2E0DC018F
:10901000ED93FC939093E6078093E5070091E507B5
:109020001091E607B8CE8AE493E00E94D9130E941B
:109030002A120E940F140E942A1210920C081092F9
:109040000B08F12CE12C2FEFE21AF20A31E0E316C3
:10905000F10441F086E493E00E94D9130E942A12A1
:109060000E940F14D801ED91FC910480F581E02D50
:10907000BE01C80119950E942A12C0900B08D09019
:109080000C080E942A12FC01868581110AC0E8148E
:10909000F9043CF4C114D10421F0F2E0CF16D1045C
:1090A00091F68EE79CE00E94F607181619062CF43C
:1090B0008EE79CE00E94D407F4CFCD2809F4F8C0D5
:1090C0005520A1F00E94001B80910609909107098C
:1090D000A0910809B09109090197A105B10531F4E2
:1090E0000E942A1221E0DC011E962C938EE393E06D
:1090F0000E94D9138CEB97E00E94D9130E942A1288
:1091000080910B0890910C080E940A14D5C0601B36
:10911000710B820B930B693873418105910508F43B
:1091200010CD0E942A12DC011E968C91882309F42E
:1091300087C086E693E00E94D9130E942A120E94FB
:109140000F140E94BA29EC01FC01E551FD4F80810A
:10915000882309F478C00E942A12CE0186579E4FB8
:109160000E949B0F6093DC087093DD088093DE08FB
:109170009093DF08FE01E451FD4F8081882309F4BC
:1091800074C00E942A12CE0186549E4F0E949B0FEB
:109190006093E0087093E1088093E2089093E308FD
:1091A000FE01E351FD4F8081882309F470C00E94C5
:1091B0002A12CE0186519E4F0E949B0F6093E408B5
:1091C0007093E5088093E6089093E7080E942A12BE
:1091D0000E94EC180E94BA290E948C190E942A123F
:1091E0000E9476120E942A120E94ED140E94001B17
:1091F0008091FE089091FF08A0910009B0910109AB
:109200000197A105B10541F08EE593E00E94D913C5
:109210000E942A120E940F148091E8089091E90898
:10922000A091EA08B091EB080196A11DB11D8093B1
:10923000E8089093E908A093EA08B093EB0877CC8C
:1092400082E693E078CF0E942A12FE01E25BFF4F94
:1092500080819181A281B3818093DC089093DD08A5
:10926000A093DE08B093DF0885CF0E942A12FE018A
:10927000E453FF4F80819181A281B3818093E00804
:109280009093E108A093E208B093E30889CF0E948D
:109290002A12C65BDE4F88819981AA81BB818093A7
:1092A000E4089093E508A093E608B093E7088ECF12
:1092B00082E493E00E94D9130E942A120E940F14A4
:1092C0000E942A1210927A0C10927B0C10927C0C45
:1092D00010927D0C4ACB5524539411113ECB0E9421
:1092E000001B8091FE089091FF08A0910009B091A9
:1092F00001090197A105B10509F426CC552009F40F
:1093000023CC82E593E00E94D9130E942A120E9486
:109310000F140E942A128FE090E090930C08809323
:109320000B0823CBEF920F931F93CF93DF93E801AA
:1093300034E047FD34E1042E000C550B57FF03C009
:10934000519541955109E32E022F242FAE01ABD147
:10935000CE01DF91CF911F910F91EF9008950F9360
:109360001F93CF93DF938230910510F482E090E059
:10937000E091BE0DF091BF0D30E020E0B0E0A0E044
:10938000309799F42115310509F44AC0281B390B8F
:1093900024303105D8F58A819B816115710589F1E9
:1093A000FB0193838283FE0111C0408151810281C0
:1093B000138148175907E0F04817590799F4109797
:1093C00061F012960C93129713961C933296CF016C
:1093D000DF91CF911F910F9108950093BE0D1093CF
:1093E000BF0DF4CF2115310551F04217530738F066
:1093F000A901DB019A01BD01DF01F801C1CFEF0135
:10940000F9CF9093BF0D8093BE0DCDCFFE01E20F3B
:10941000F31F819391932250310939832883D7CF49
:109420002091BC0D3091BD0D232B41F420910402FD
:10943000309105023093BD0D2093BC0D20910202A6
:10944000309103022115310541F42DB73EB740910B
:10945000060250910702241B350BE091BC0DF091E0
:10946000BD0DE217F307A0F42E1B3F0B2817390799
:1094700078F0AC014E5F5F4F2417350748F04E0F70
:109480005F1F5093BD0D4093BC0D819391939FCF6F
:10949000F0E0E0E09CCFCF93DF930097E9F0FC0190
:1094A000329713821282A091BE0DB091BF0DED01D3
:1094B00030E020E01097A1F420813181820F931FCA
:1094C0002091BC0D3091BD0D2817390709F061C0FE
:1094D000F093BD0DE093BC0DDF91CF910895EA01AB
:1094E000CE17DF07E8F54A815B819E0141155105E2
:1094F000B1F7E901FB83EA8349915991C40FD51F64
:10950000EC17FD0761F4808191810296840F951F0D
:10951000E90199838883828193819B838A83F0E028
:10952000E0E012968D919C9113970097B9F52D91DB
:109530003C911197CD010296820F931F2091BC0D93
:109540003091BD0D2817390739F6309751F5109233
:10955000BF0D1092BE0DB093BD0DA093BC0DBCCF3E
:10956000D383C28340815181840F951FC817D907C7
:1095700061F44E5F5F4F88819981480F591F518375
:1095800040838A819B81938382832115310509F071
:10959000B0CFF093BF0DE093BE0D9ECFFD01DC0177
:1095A000C0CF13821282D7CF66277727F4C14AEB48
:1095B0005DE000C0FA01A191B081009719F4109705
:1095C000E1F0CD01DC01CD010D90002011F4C001CE
:1095D00013C0FB012191222319F02015D9F7F3CFF5
:1095E000FB012191201519F41E92119606C0222329
:1095F000C1F70D900020A1F7D001FA01A193B0832B
:109600000895BB274A3031F4992322F4BDE29095A6
:1096100081959F4F30C0BB272A3051F4992342F4E3
:10962000BDE290958095709561957F4F8F4F9F4FCC
:1096300001C0BB27FA01A62F6217710581059105AC
:10964000330B30FB66F0AA27660F771F881F991F20
:10965000AA1FA21710F0A21B63953850A9F7A05DAE
:10966000AA3308F0A95DA19336F7B111B193108226
:10967000CA01DEC3BB27FB015527AA27880F991F04
:10968000AA1FA41710F0A41B83955051B9F7A05D31
:10969000AA3308F0A95DA193009779F7B111B193AE
:1096A0001192CB01C5C38F929F92AF92BF92CF927E
:1096B000DF92EF92FF920F931F93CF93DF9300D02F
:1096C00000D000D0CDB7DEB76A01F22EB02E102F39
:1096D000FBE3AF2EA01608F41BE31F5F012F27E06A
:1096E000AE014F5F5F4FACD2BC018981982F99705A
:1096F000913009F44EC09BE2E1FC04C09E2D9170B4
:10970000E0FC49C05E2D5071E82FE87083FF55C022
:1097100084E0911101C083E0EF2DE81B8F1508F064
:10972000E0E0D6018E2F20E25523C9F1992329F0DC
:10973000D6019C93C60101966C0196012D5F3F4FA7
:10974000E2FE33C08EE4D6018C9391E411969C9393
:10975000119712968C93D9018E2F90E281112AC015
:10976000E20FF32FF11D10828EEF9FEF29960FB6B7
:10977000F894DEBF0FBECDBFDF91CF911F910F9147
:10978000FF90EF90DF90CF90BF90AF909F908F9021
:1097900008959DE2B7CF90E2B5CF2D93815081110E
:1097A000FCCFCE0ED11CE0E0C1CF8EE6D6018C936B
:1097B00091E6CCCF9D938150D1CF482F447082FF4A
:1097C0003DC084E0911101C083E08F1510F4EF2DAE
:1097D000E81BD6018E2F20E2552309F1992329F0A9
:1097E000D6019C93C60101966C0196012D5F3F4FF7
:1097F000E2FE1BC089E4D6018C938EE411968C9313
:10980000119786E412968C93D9018E2F90E28823CB
:1098100009F4A6CF9D938150FACF2D9381508111E9
:10982000FCCFCE0ED11CE0E0D9CF89E6D6018C93D7
:109830008EE611968C93119786E6E4CF9B0177FF15
:1098400002C030E020E0A1E0B0E0911102C0B0E041
:10985000A0E0F9013196AE0FBF1F8B2C912CBB20DD
:1098600009F461C05401EFEFAE1ABE0AAA0DBB1D88
:10987000FA161B0619F014F04F2D4A1B511188C01F
:10988000E3FC59C07601A42FB0E2A1114FC0C40E71
:10989000D11C992309F45BC040E0D6011196F60172
:1098A00090836D01552309F448C0012F060F9A815A
:1098B000582F507184FF03C0913309F401501016E2
:1098C0000CF047C0093008F008E0EEE2FE2E5B0124
:1098D000A01AB10885019194819491082F3F320715
:1098E00029F4D601FC92F60131966F0162177307D5
:1098F00094F1021713077CF5DB01A21BB30BAA241A
:10990000A394B12CAC0EBD1EAA0DBB1D11968C915B
:1099100021503109D601119628153905F4F0F601C8
:1099200080836D01DBCFB12CA12CA0CFF701B193C7
:109930007F01A150AACF9111B0CFD601942F50E34F
:1099400002C05D9391509111FCCFC40ED11C40E038
:10995000ACCF01E0BACF80E3DBCF6217730731F4FD
:10996000963388F4953311F4552369F0F60180831A
:10997000FD01842F90E2811108C0A40FB11D1C923B
:1099800090E080E0F3CE81E3F1CF91938150F3CF6B
:10999000911183CF8ACF8F929F92AF92BF92CF9235
:1099A000DF92EF92FF920F931F93CF93DF935C01AF
:1099B0007B016115710519F0DB018D939C93850185
:1099C0000F5F1F4FF501D0818D2F90E011D26C01F8
:1099D000892BA9F5DD32A9F50F5F1F4FD50111962F
:1099E000DC91C1E05801F1E0AF1AB10843E050E06A
:1099F0006CEE70E0C50104D2892B61F5680182E04C
:109A0000C80ED11C45E050E067EE70E0C601F8D109
:109A1000892B21F4680197E0C90ED11CE114F104EF
:109A200019F0D701CD92DC9260E070E080E89FEF02
:109A3000C111F9C060E070E080E89FE7F4C0580110
:109A4000BECFDB3229F485010E5F1F4FF501D181B6
:109A5000C0E0C8CF43E050E064EE70E0C501D0D173
:109A6000892BE9F0F80110E000E020E030E0A901E6
:109A70005F01B0ED8B2E8D0E89E08815C0F19C2E14
:109A8000689491F88C2F8870C2FF16C0811102C0B3
:109A90000F5F1F4F3196D501DC91C92DE9CFE1143D
:109AA000F10429F00E5F1F4FF7011183008360E07E
:109AB00070E080EC9FE7B7C0882311F001501109D6
:109AC000A5E0B0E013D39B01AC01220F331F441F6C
:109AD000551F280D311D411D511D283999E93907A0
:109AE000490799E15907B0F2C6609C2ED3CFAEEF7B
:109AF0008A1206C0C3FD3CC09C2E689493F8CACF5E
:109B0000DF7DD534A9F580818D3239F4C061DF0164
:109B10001296818162E070E006C0DF018B32C1F3F2
:109B2000119661E070E080535D01A61AB70A8A3091
:109B3000F8F4E0E8CE16ECE0DE065CF4B601660F61
:109B4000771F660F771FC60ED71ECC0CDD1CC80E04
:109B5000D11C5D01FFEFAF1ABF0A8C9180538A3090
:109B600098F1C4FF03C0D194C194D1080C0D1D1D00
:109B7000C1FF09C0E114F10431F081E0A81AB10875
:109B8000D701AD92BC92CA01B90166D1C370C3308E
:109B900009F490584B015C0120E030E0A90158D154
:109BA000882309F43EC0CBE1D1E017FF05C0119531
:109BB00001951109C3E0D1E06E01B8E1CB1AD108DB
:109BC00080E2E82EF12C0EC0D501B3CFFE01259125
:109BD0003591459154910E191F09C501B4019DD1CC
:109BE0004B015C01D501C4010E151F057CF72497BC
:109BF000F594E794CC16DD06A9F78A2F880F8B2FF2
:109C0000881F8F3F41F020E030E0A901C501B40179
:109C10001FD1811106C082E290E09093C10D809324
:109C2000C00DC501B401DF91CF911F910F91FF903D
:109C3000EF90DF90CF90BF90AF909F908F9008955E
:109C4000283008F027E03327DA01990F311D87FD0E
:109C5000916000966105710539F432602E5F3D9385
:109C600030E32A95E1F708959F3F30F08038710581
:109C7000610509F03C5F3C5F3D93913008F08068DE
:109C8000911DDF93CF931F930F93FF92EF92192FA4
:109C9000987F9695E92F96959695E90FFF27E758B7
:109CA000FE4F99273327EE24FF24A701E7010590F3
:109CB0000894079428F4360FE71EF81E491F511D1B
:109CC000660F771F881F991F0694A1F705900794C8
:109CD00028F4E70EF81E491F561FC11D770F881F75
:109CE000991F661F0694A1F70590079428F4F80EB3
:109CF000491F561FC71FD11D880F991F661F771F49
:109D00000694A1F70590079420F4490F561FC71F2A
:109D1000D81F990F661F771F881F0694A9F7849193
:109D20001095177041F0D695C79557954795F794BC
:109D3000E7941A95C1F7EFE1F1E068941590159159
:109D400035916591959105907FE27395E118F10A3F
:109D5000430B560BC90BD009C0F7E10CF11E431F92
:109D6000561FC91FD01D7EF4703311F48A95E6CFBB
:109D7000E894015030F0080F0AF40027021708F4A5
:109D8000202F2395022F7A3328F079E37D932A95AB
:109D9000E9F710C07D932A9589F606949795679503
:109DA000379517951794E118F10A430B560BC90B19
:109DB000D00998F023957E9173957A3308F070E37B
:109DC0007C932013B8F77E9170617D9330F083957A
:109DD00071E37D9370E32A95E1F71124EF90FF90F2
:109DE0000F911F91CF91DF91992787FD909508954D
:109DF0009111F6C0803219F089508550D0F708953E
:109E0000FB01DC014150504088F08D9181341CF001
:109E10008B350CF4805E659161341CF06B350CF46D
:109E2000605E861B611171F3990B0895881BFCCF4E
:109E3000DC01FC01672F71917723E1F7329704C0B1
:109E40007C916D9370836291AE17BF07C8F308953C
:109E500040D008F481E00895E89409C097FB3EF4EF
:109E600090958095709561957F4F8F4F9F4F992367
:109E7000A9F0F92F96E9BB279395F69587957795E5
:109E80006795B795F111F8CFFAF4BB0F11F460FFA5
:109E90001BC06F5F7F4F8F4F9F4F16C0882311F0FD
:109EA00096E911C0772321F09EE8872F762F05C011
:109EB000662371F096E8862F70E060E02AF09A95AC
:109EC000660F771F881FDAF7880F9695879597F9A1
:109ED0000895990F0008550FAA0BE0E8FEEF16163B
:109EE0001706E807F907C0F012161306E407F5078E
:109EF00098F0621B730B840B950B39F40A2661F002
:109F0000232B242B252B21F408950A2609F4A140A4
:109F1000A6958FEF811D811D08950BD07BC06CD05D
:109F200028F071D018F0952309F05DC062C01124AB
:109F3000A5C081D0A0F3959FD1F3950F50E0551F98
:109F4000629FF001729FBB27F00DB11D639FAA278E
:109F5000F00DB11DAA1F649F6627B00DA11D661FDD
:109F6000829F2227B00DA11D621F739FB00DA11DFE
:109F7000621F839FA00D611D221F749F3327A00DB8
:109F8000611D231F849F600D211D822F762F6A2F54
:109F900011249F5750408AF0E1F088234AF0EE0FD9
:109FA000FF1FBB1F661F771F881F91505040A9F7E6
:109FB0009E3F510570F017C061C05F3FECF3983EC3
:109FC000DCF3869577956795B795F795E7959F5F4D
:109FD000C1F7FE2B880F911D9695879597F90895E7
:109FE00099278827089597F99F6780E870E060E0D7
:109FF00008959FEF80EC089500240A941616170622
:10A0000018060906089500240A9412161306140669
:10A0100005060895092E0394000C11F4882352F0CC
:10A02000BB0F40F4BF2B11F460FF04C06F5F7F4F84
:10A030008F4F9F4F089557FD9058440F551F59F06B
:10A040005F3F71F04795880F97FB991F61F09F3F25
:10A0500079F087950895121613061406551FF2CF4E
:10A060004695F1DF08C0161617061806991FF1CF9E
:10A0700086957105610508940895E894BB276627C5
:10A080007727CB0197F90895F999FECF92BD81BD4D
:10A09000F89A992780B50895262FF999FECF1FBA0F
:10A0A00092BD81BD20BD0FB6F894FA9AF99A0FBE01
:10A0B00001960895052E97FB16F400940FD057FDD6
:10A0C00005D024D007FC02D046F408C05095409536
:10A0D000309521953F4F4F4F5F4F08959095809554
:10A0E000709561957F4F8F4F9F4F089531D0A59FF9
:10A0F000900DB49F900DA49F800D911D1124089583
:10A10000B7FFF4CFF3DF821B930B0895A1E21A2E61
:10A11000AA1BBB1BFD010DC0AA1FBB1FEE1FFF1F0B
:10A12000A217B307E407F50720F0A21BB30BE40B5B
:10A13000F50B661F771F881F991F1A9469F76095A2
:10A140007095809590959B01AC01BD01CF0108955C
:10A15000A29FB001B39FC001A39F700D811D112468
:10A16000911DB29F700D811D1124911D08955058AD
:10A17000BB27AA270ED04ECF3FDF30F044DF20F0C0
:10A1800031F49F3F11F41EF434CF0EF4E095E7FB59
:10A190002ACFE92F50DF80F3BA17620773078407CD
:10A1A000950718F071F49EF568CF0EF4E0950B2E2C
:10A1B000BA2FA02D0B01B90190010C01CA01A00119
:10A1C0001124FF27591B99F0593F50F4503E68F174
:10A1D0001A16F040A22F232F342F4427585FF3CFB5
:10A1E000469537952795A795F0405395C9F77EF486
:10A1F0001F16BA0B620B730B840BBAF09150A1F0CF
:10A20000FF0FBB1F661F771F881FC2F70EC0BA0F54
:10A21000621F731F841F48F4879577956795B795DC
:10A22000F7959E3F08F0B3CF9395880F08F09927D4
:10A23000EE0F9795879508950CD0ECCEE4DE40F0B4
:10A24000DBDE30F021F45F3F19F0CDCE511116CF97
:10A25000D0CEF1DE98F39923C9F35523B1F3951BC2
:10A26000550BBB27AA2762177307840738F09F5F37
:10A270005F4F220F331F441FAA1FA9F333D00E2EA6
:10A280003AF0E0E830D091505040E695001CCAF713
:10A2900029D0FE2F27D0660F771F881FBB1F2617D8
:10A2A00037074807AB07B0E809F0BB0B802DBF01AB
:10A2B000FF2793585F4F2AF09E3F510568F093CED9
:10A2C000DDCE5F3FECF3983EDCF38695779567959E
:10A2D000B795F7959F5FC9F7880F911D969587955C
:10A2E00097F90895E1E0660F771F881FBB1F62177B
:10A2F00073078407BA0720F0621B730B840BBA0B39
:10A30000EE1F88F7E095089504D06894B111B6CE99
:10A31000089599DE88F09F5790F0B92F9927B7518B
:10A32000A0F0D1F0660F771F881F991F1AF0BA9519
:10A33000C9F712C0B13081F0A0DEB1E008959DCE22
:10A34000672F782F8827B85F39F0B93FCCF386950F
:10A3500077956795B395D9F73EF49095809570956C
:10A3600061957F4F8F4F9F4F0895B3DD08F48FEFB6
:10A370000895AFDD880B990B0895DB018F939F93B0
:10A38000B5DEBF91AF91A29F800D911DA39F900D4F
:10A39000B29F900D11240895991B79E004C0991F74
:10A3A000961708F0961B881F7A95C9F7809508952F
:10A3B000EE0FFF1F881F8BBF0790F691E02D1994B9
:10A3C0004F925F926F927F928F929F92AF92BF92C5
:10A3D000CF92DF92EF92FF920F931F93CF93DF9371
:10A3E0008C01009799F4CB01DF91CF911F910F91D0
:10A3F000FF90EF90DF90CF90BF90AF909F908F90A5
:10A400007F906F905F904F900C94AF49FC01E60FE6
:10A41000F71F9C0122503109E217F30708F4ACC082
:10A42000D901CD91DC911197C617D70718F1C53026
:10A43000D10570F0CE0104978617970748F0C61B28
:10A44000D70B2297C193D1936D937C93CF0123D8DF
:10A45000C801DF91CF911F910F91FF90EF90DF9096
:10A46000CF90BF90AF909F908F907F906F905F90B4
:10A470004F9008955B01AC1ABD0A4C018C0E9D1ED5
:10A48000A091BE0DB091BF0D512C412CF12CE12CAF
:10A49000109731F58091BC0D9091BD0D88159905EF
:10A4A00009F05CC04616570608F058C080910202B9
:10A4B00090910302009741F48DB79EB74091060238
:10A4C00050910702841B950BE817F90708F054C058
:10A4D000F093BD0DE093BC0DF90171836083B8CF9B
:10A4E0008D919C91119712966C90129713967C9077
:10A4F0001397A815B90559F56C0142E0C40ED11C9B
:10A50000CA14DB0420F1AC014A195B09DA01129686
:10A51000159780F06282738251834083D9016D93D5
:10A520007C93E114F10471F0D7011396FC93EE9340
:10A5300012978ECF22968C0F9D1FF90191838083F5
:10A54000F301EFCFF093BF0DE093BE0D81CF48161E
:10A55000590608F42C017D01D3019ACFCB010E944A
:10A56000AF497C01009741F0AE01B80108D0C801A5
:10A570000E944B4A87016CCF10E000E069CFFB01DD
:10A58000DC0102C001900D9241505040D8F708956F
:10A59000FB01DC018D91019080190110D9F3990B19
:10A5A0000895FB01DC0101900D920020E1F7089570
:04A5B000F894FFCF4D
:10A5B400FFFF0000C20D8000362E352E302E5200D3
:10A5C40000010000000100000001000000200A0D4D
:10A5D40000005238350052383400523035005231C0
:10A5E4003300523132005231310052373300523786
:10A5F4003200523731005231370052313600523175
:10A60400350052303400523837000D0A0020005211
:10A614003939000D0A0020005239390000000000C9
:10A624003910F0262A2A000000002612FA263915CD
:10A6340000000000380FE6268719000000003710DC
:10A64400EC26171500000000330FE026CE120000A0
:10A6540000004711F6263F13000000003610EA26DA
:10A66400321300000000320FDE26DF140000000069
:10A674002912FE267913000000002512F826702600
:10A68400000000002812FC26BC2600000000ED0B90
:10A69400D426731B00000000EE0BD626AE38000053
:10A6A40000002712D226C53B000000003311F22619
:10A6B4008C3B000000003810EE26E63A0000000053
:10A6C400EF0BD826E73800000000370FE4261E3AC7
:10A6D40000000000310FDC26B51200000000F00B72
:10A6E400DA267339000000003510E826AA3A523001
:10A6F4003300523032005230370052303100523081
:10A704003900523838005238370052303800523845
:10A7140038005230300052383700523036000000D2
:10A7240000002D089807C5077D08F607D407E80739
:10A7340000000000EC0BF42620510052343100508C
:10A74400005238310020584100205842002059411D
:10A754000020594200205A4100205A4200686F6D7F
:10A76400650D0A0052383320005232310052393913
:10A77400204572726F723A20696E76616C6964204A
:10A78400706172616D657465722069640D0A0052AE
:10A794003939002073746120002063757220002011
:10A7A400656E6420002068616C662000206C656E14
:10A7B4002000206D696E2000206D617820002073D8
:10A7C400706420006E616E00696E66006F766600CC
:10A7D40052383200523230005239392057696C6C89
:10A7E400207A65726F2058005239392057696C6C91
:10A7F400207A65726F2059005239392057696C6C80
:10A80400207A65726F205A005239392043616C698D
:10A8140062726174696F6E206572726F723A20653C
:10A824006E642073746F702061637469766520624E
:10A8340065666F72652073746172740D0A0020611D
:10A844007869732000206D6F766520746F207374AF
:10A8540061727420666F722063616C6962726174E4
:10A86400696F6E0052393920656D657267656E6374
:10A87400792073746F700D0A00523939206D6F7628
:10A88400656D656E7420646F6E650D0A00206174D9
:10A89400207374617274696E6720706F696E7400DE
:10A8A400523233002063616C6962726174696E674D
:10A8B400206C656E67746800207374657020636F24
:10A8C400756E743A200020617420656E6420706F88
:10A8D400696E7400206465616374697661746520CF
:10A8E4006D6F746F7220582064756520746F206DCD
:10A8F40069737365642073746570730020646561A3
:10A9040063746976617465206D6F746F7220592069
:10A9140064756520746F206D697373656420737446
:10A924006570730020646561637469766174652081
:10A934006D6F746F72205A2064756520746F206D7A
:10A9440069737365642073746570730052393920B8
:10A9540074696D656F7574205820617869730D0A88
:10A96400005239392074696D656F757420592061FE
:10A974007869730D0A005239392074696D656F75F1
:10A9840074205A20617869730D0A005239392065A0
:10A9940072726F720D0A005239392073746F7070BD
:10A9A40065640D0A00523939206572726F72200095
:10A9B40053657269616C20636F6E6E656374696F51
:10A9C4006E20737461727465640053657420696EDB
:10A9D4007075742F6F75747075740052656164209E
:10A9E400706172616D6574657273004C6F6164208F
:10A9F4006D6F76656D656E742073657474696E67CA
:10AA04007300536574206D6F746F7220656E61629C
:10AA14006C6573206F66660053746172742070698C
:10AA24006E2067756172640053746172742073657B
:10AA340072766F00537461727420696E74657272F9
:10AA440075707400436865636B20686F6D696E6729
:10AA5400206F6E20626F6F740052393920484F4D59
:10AA640045205A204F4E20535441525455500D0AFC
:10AA74000052393920484F4D452059204F4E20531C
:10AA84005441525455500D0A0052393920484F4D03
:10AA9400452058204F4E20535441525455500D0ACE
:10AAA4000041524455494E4F20535441525455503D
:10AAB40020434F4D504C455445002A004730004731
:10AAC40030300047310047303100473238004630DB
:10AAD40039004639004631310046313200463133BF
:10AAE40000463134004631350046313600463230B6
:10AAF40000463231004632320046333100463332AA
:10AB0400004634310046343200463433004634348F
:10AB14000046363100463831004638320046383374
:10AB24000046383400200A0D005239392068616E1D
:10AB3400646C6572203D3D204E554C4C0D0A00203E
:10AB4400726573657474696E67206469676974619A
:10AB54006C2070696E0020726573657474696E6729
:10AB640020616E616C6F672070696E002056000072
:00000001FF
